:030000000262DCBD
:1062DC00758E1190000078FF79FFE4F0A3D9FBD8FC
:0D62EC00F778FFE4F6D8FD75816B0263348E
:106722004401D240490FDB4401CE40C90FDB440192
:05673200CA3C8EFA359F
:064389009001B2121F5E5C
:10438F009001B6E0FCA3E0FDA3E0FEA3E0FFEF2465
:10439F0069FFEE3474FEED34FFFDEC34FFFCEC12DC
:1043AF001AC87BDF7A927986783D1218A49001BAE9
:1043BF00121F5E7B007A0079C078419001BAE0FC51
:1043CF00A3E0FDA3E0FEA3E0FF1219AD125A647B38
:1043DF00007A0079C078411218A4C004C005C00645
:1043EF00C0077F977E7E7DD57C409001BAE0F8A311
:1043FF00E0F9A3E0FAA3E0FB1217B3D003D002D089
:10440F0001D0001217AFC004C005C006C0077F92CD
:10441F007E867DC07C419001B2E0F8A3E0F9A3E075
:10442F00FAA3E0FB1218A4A804A905AA06AB07D0AB
:10443F0007D006D005D0041217B39001C2121F5E29
:10444F009001B6E0FCA3E0FDA3E0FEA3E0FFEF24A4
:10445F0069FFEE3474FEED34FFFDEC34FFFCEC121B
:10446F001AC89001B2E0F8A3E0F9A3E0FAA3E0FBC9
:10447F001217B37B307AE67958783D1218A4A80446
:10448F00A905AA06AB077F817E0E7DBA7C43121762
:10449F00AF9001CAE0F8A3E0F9A3E0FAA3E0FB12A2
:1044AF0018A49001BE121F5E9001CEE0FCA3E0FDA8
:1044BF00A3E0FEA3E0FF9001BEE0F8A3E0F9A3E0C4
:1044CF00FAA3E0FB121A4A602940279001BEE0FCD4
:1044DF00A3E0FDA3E0FEA3E0FF9001CEE0F8A3E090
:1044EF00F9A3E0FAA3E0FB1217AF9001BE121F5E13
:1044FF0080B69001CEE0FCA3E0FDA3E0FEA3E0FFB9
:10450F00121AB79001BEE0F8A3E0F9A3E0FAA3E016
:10451F00FB121A4A50279001BEE0FCA3E0FDA3E076
:10452F00FEA3E0FF9001CEE0F8A3E0F9A3E0FAA329
:10453F00E0FB1217B39001BE121F5E80B57F007EA5
:10454F00007D007C009001BEE0F8A3E0F9A3E0FA43
:10455F00A3E0FB121A4A604840469001D2E0FCA348
:10456F00E0FDA3E0FEA3E0FF9001BEE0F8A3E0F9B9
:10457F00A3E0FAA3E0FB121A4A50259001BEE0FC1B
:10458F00A3E0FDA3E0FEA3E0FF9001CEE0F8A3E0DF
:10459F00F9A3E0FAA3E0FB1217AF9001BE121F5E62
:1045AF007F007E007D007C009001BEE0F8A3E0F963
:1045BF00A3E0FAA3E0FB121A4A504B9001D2E0FCA1
:1045CF00A3E0FDA3E0FEA3E0FF121AB79001BEE047
:1045DF00F8A3E0F9A3E0FAA3E0FB121A4A60274020
:1045EF00259001BEE0FCA3E0FDA3E0FEA3E0FF9059
:1045FF0001CEE0F8A3E0F9A3E0FAA3E0FB1217B3B2
:10460F009001BE121F5E9001BEE0FCA3E0FDA3E08F
:10461F00FEA3E0FF1252747B247A0B79987839123B
:10462F0018A49001C2E0F8A3E0F9A3E0FAA3E0FB1D
:10463F001217B39001C6121F5E7B007A0079C07803
:10464F00419001C6E0FCA3E0FDA3E0FEA3E0FF1252
:10465F0019AD125A647B007A0079C078411218A400
:10466F00A804A905AA06AB079001C6E0FCA3E0FDCC
:09467F00A3E0FEA3E0FF1217AF57
:01468800220F
:1066E0009001DB121F5E9001DBE0FCA3E0FDA3E064
:1066F000FEA3E0FF125A64A804A905AA06AB0790FE
:1067000001DBE0FCA3E0FDA3E0FEA3E0FF1217AF76
:106710009001CEE0F8A3E0F9A3E0FAA3E0FB1218A1
:02672000A422B1
:060C7D00900142121F5E0F
:100C8300900142E0FCA3E0FDA3E0FEA3E0FFEF241C
:100C930013FFEE342DFEED34FFFDEC34FFFCEC12BC
:100CA3001AC8900146E0F8A3E0F9A3E0FAA3E0FB39
:100CB3001217B390014A121F5E7F8D7EA67D147CAE
:100CC3003D90014AE0F8A3E0F9A3E0FAA3E0FB12A8
:100CD30018A47B807AF279BF783E1217B31266E0CC
:100CE30090014E121F5E7F477E857D167C3D9001ED
:100CF3004AE0F8A3E0F9A3E0FAA3E0FB1218A47B0F
:100D0300937AA77984783E1217B31266E090015262
:100D1300121F5E7F217EB47D0A7C3D90014AE0F87C
:100D2300A3E0F9A3E0FAA3E0FB1218A47BFF7ACDBA
:100D33007953783F1217B31266E0900156121F5E83
:100D43007F4D7E6C7D337C3B90014AE0F8A3E0F954
:100D5300A3E0FAA3E0FB1218A47B817A3D797E78A5
:100D63003F1217B31266E090015A121F5E7F007E96
:100D7300007D007C40900156E0F8A3E0F9A3E0FA7F
:100D8300A3E0FB1218A4A804A905AA06AB079001C7
:100D93004EE0FCA3E0FDA3E0FEA3E0FF1217AF12B9
:100DA300525E7BF37A767914783F1218A4C004C09C
:100DB30005C006C00790014EE0FCA3E0FDA3E0FEE2
:100DC300A3E0FF12525E7BE87AC179517840121892
:100DD300A4A804A905AA06AB077FB17E737D717C25
:100DE300421217AFD003D002D001D0001217AFC008
:100DF30004C005C006C0077F007E007D007C4090D4
:100E03000156E0F8A3E0F9A3E0FAA3E0FB1218A46B
:100E130012525E7B0C7A5979ED783E1218A4A8041D
:100E2300A905AA06AB07D007D006D005D004121730
:100E3300AF90015E121F5E7F007E007D007C4090BC
:100E43000156E0F8A3E0F9A3E0FAA3E0FB1218A42B
:100E5300C004C005C006C0077F007E007D007C4043
:100E630090014EE0F8A3E0F9A3E0FAA3E0FB121827
:100E7300A4D003D002D001D0001217AF12525E7B70
:100E8300767A4F791E783D1218A4C004C005C006B7
:100E9300C0077F007E007D007C4090014EE0F8A3F8
:100EA300E0F9A3E0FAA3E0FB1218A412525E7B9CC4
:100EB3007A5A79B6783D1218A4A804A905AA06ABF4
:100EC3000790015EE0FCA3E0FDA3E0FEA3E0FF12B8
:100ED30017AFA804A905AA06AB07D007D006D0050B
:100EE300D0041217B3C004C005C006C0077F007E3C
:100EF300007D007C40900156E0F8A3E0F9A3E0FAFE
:100F0300A3E0FB1218A490015AE0F8A3E0F9A3E0D0
:100F1300FAA3E0FB1217AF12525E7B687A9679044C
:100F2300783D1218A4A804A905AA06AB07D007D0D8
:100F330006D005D0041217AF90015E121F5E7F002A
:100F43007E007D007C40900156E0F8A3E0F9A3E029
:100F5300FAA3E0FB1218A4A804A905AA06AB0790FC
:100F6300014EE0FCA3E0FDA3E0FEA3E0FF1217AFF8
:100F730090015AE0F8A3E0F9A3E0FAA3E0FB12170B
:100F8300B312525E7BD87A2A79C1783C1218A4C076
:100F930004C005C006C0077F007E007D007C409032
:100FA3000156E0F8A3E0F9A3E0FAA3E0FB1218A4CA
:100FB300A804A905AA06AB0790014EE0FCA3E0FD37
:100FC300A3E0FEA3E0FF1217AF12525E7B727A33E7
:100FD30079DC783C1218A4A804A905AA06AB0790EB
:100FE300015EE0FCA3E0FDA3E0FEA3E0FF1217AF68
:100FF300D003D002D001D0001217AFC004C005C087
:1010030006C00790015AE0F8A3E0F9A3E0FAA3E0D1
:10101300FB90014EE0FCA3E0FDA3E0FEA3E0FF1282
:1010230017AF12525E7B307A4C79A6783C1218A423
:10103300A804A905AA06AB07D007D006D005D0049B
:101043001217AF90015E121F5E900156E0FCA3E001
:10105300FDA3E0FEA3E0FF12525E7B0B7AD2798CF4
:10106300783C1218A490015EE0F8A3E0F9A3E0FA3B
:10107300A3E0FB1217B3C004C005C006C00790016C
:101083005AE0FCA3E0FDA3E0FEA3E0FF90014EE0E5
:10109300F8A3E0F9A3E0FAA3E0FB1217B312525E40
:1010A3007B697AE37988783C1218A4A804A905AA75
:1010B30006AB07D007D006D005D0041217B39001B2
:1010C3005E121F5E7F007E007D007C40900152E037
:1010D300F8A3E0F9A3E0FAA3E0FB1218A4A804A97B
:1010E30005AA06AB0790014EE0FCA3E0FDA3E0FEDA
:1010F300A3E0FF1217AF12525E7BF97A4E794C7858
:101103003C1218A4C004C005C006C00790015AE0F1
:10111300FCA3E0FDA3E0FEA3E0FF12525E7BCD7AC9
:10112300AF79E6783B1218A4A804A905AA06AB0771
:10113300D007D006D005D0041217B3C004C005C031
:1011430006C0077F007E007D007C40900156E0F8DA
:10115300A3E0F9A3E0FAA3E0FB1218A490015AE07C
:10116300F8A3E0F9A3E0FAA3E0FB1217B312525E6F
:101173007BBC7A5779AD783B1218A4A804A905AAB9
:1011830006AB07D007D006D005D0041217B3C004AE
:10119300C005C006C0077F007E007D807C409001B3
:1011A30056E0F8A3E0F9A3E0FAA3E0FB1218A4A821
:1011B30004A905AA06AB0790014EE0FCA3E0FDA33A
:1011C300E0FEA3E0FF1217AF12525E7B4E7AB479B2
:1011D300AB783B1218A4A804A905AA06AB07D0074D
:1011E300D006D005D0041217AF900162121F5E7FA4
:1011F300007E007D007C40900156E0F8A3E0F9A357
:10120300E0FAA3E0FB1218A4A804A905AA06AB07F9
:1012130090014EE0FCA3E0FDA3E0FEA3E0FF121764
:10122300AF90015AE0F8A3E0F9A3E0FAA3E0FB12C0
:1012330017AF12525E7BA97A6A7982783B1218A49F
:10124300900162E0F8A3E0F9A3E0FAA3E0FB121730
:10125300B3C004C005C006C0077F007E007D407C8C
:101263004090014EE0F8A3E0F9A3E0FAA3E0FB12FB
:1012730018A412525E7B9C7ADC796F783B1218A417
:10128300A804A905AA06AB07D007D006D005D00449
:101293001217AFC004C005C006C0077F007E007DE3
:1012A300807C40900156E0F8A3E0F9A3E0FAA3E0C4
:1012B300FB1218A4C004C005C006C0077F007E004F
:1012C3007D007C4090014EE0F8A3E0F9A3E0FAA38F
:1012D300E0FB1218A4D003D002D001D0001217AF44
:1012E30012525E7BCA7A547941783B1218A4A8043F
:1012F300A905AA06AB07D007D006D005D00412175C
:10130300AF900162121F5E7F007E007D007C4090E3
:101313000156E0F8A3E0F9A3E0FAA3E0FB1218A456
:10132300C004C005C006C0077F007E007D407C402E
:1013330090014EE0F8A3E0F9A3E0FAA3E0FB121852
:10134300A4D003D002D001D0001217AF12525E7B9B
:10135300457A2F7923783B1218A4C004C005C00630
:10136300C00790015AE0FCA3E0FDA3E0FEA3E0FF69
:10137300900156E0F8A3E0F9A3E0FAA3E0FB12170B
:10138300B312525E7B147A5C792C783B1218A4A8B2
:1013930004A905AA06AB07900162E0FCA3E0FDA344
:1013A300E0FEA3E0FF1217AFA804A905AA06AB0746
:1013B300D007D006D005D0041217B3C004C005C0AF
:1013C30006C0077F007E007D007C40900156E0F858
:1013D300A3E0F9A3E0FAA3E0FB1218A490014EE006
:1013E300F8A3E0F9A3E0FAA3E0FB1217B390015AC4
:1013F300E0F8A3E0F9A3E0FAA3E0FB1217AF12525F
:101403005E7BA67AD57910783B1218A4A804A905A7
:10141300AA06AB07D007D006D005D0041217AFC079
:1014230004C005C006C0077F007E007D007C40909D
:101433000156E0F8A3E0F9A3E0FAA3E0FB1218A435
:10144300C004C005C006C0077F007E007D007C404D
:10145300900152E0F8A3E0F9A3E0FAA3E0FB12182D
:10146300A4D003D002D001D0001217AF12525E7B7A
:10147300B37A7B79F2783A1218A4A804A905AA06CC
:10148300AB07D007D006D005D0041217B390016282
:10149300121F5E7F007E007D007C40900152E0F8C9
:1014A300A3E0F9A3E0FAA3E0FB1218A490014EE035
:1014B300F8A3E0F9A3E0FAA3E0FB1217B3C004C05A
:1014C30005C006C0077F007E007D007C409001566A
:1014D300E0F8A3E0F9A3E0FAA3E0FB1218A4A80440
:1014E300A905AA06AB07D007D006D005D00412176A
:1014F300AF12525E7B047AAD79C0783A1218A4C059
:1015030004C005C006C0077F007E007D007C4090BC
:10151300015AE0F8A3E0F9A3E0FAA3E0FB1218A450
:10152300C004C005C006C0077F007E007D007C406C
:10153300900156E0F8A3E0F9A3E0FAA3E0FB121848
:10154300A4D003D002D001D0001217AF12525E7B99
:10155300A37A0679D378BA1218A4A804A905AA060F
:10156300AB07D007D006D005D0041217B3C004C010
:1015730005C006C0077F007E007D807C4090015639
:10158300E0F8A3E0F9A3E0FAA3E0FB1218A41252D7
:101593005E7B4B7A1F79BA783A1218A4A804A9057E
:1015A300AA06AB07D007D006D005D0041217AFC0E8
:1015B30004C005C006C0077F007E007D007C40900C
:1015C3000156E0F8A3E0F9A3E0FAA3E0FB1218A4A4
:1015D300C004C005C006C0077F007E007D007C40BC
:1015E30090014EE0F8A3E0F9A3E0FAA3E0FB1218A0
:1015F300A4D003D002D001D0001217AF90015AE05B
:10160300F8A3E0F9A3E0FAA3E0FB1217B312525ECA
:101613007BA97A3079B6783A1218A4A804A905AA46
:1016230006AB07D007D006D005D0041217B390013C
:1016330066121F5E7F007E007D807C40900156E035
:10164300F8A3E0F9A3E0FAA3E0FB1218A4A804A905
:1016530005AA06AB0790014EE0FCA3E0FDA3E0FE64
:10166300A3E0FF1217AF90015AE0F8A3E0F9A3E05B
:10167300FAA3E0FB1217B312525E7B3B7AAA799A64
:10168300783A1218A4A804A905AA06AB0790016624
:10169300E0FCA3E0FDA3E0FEA3E0FF1217AFC0044C
:1016A300C005C006C0077F007E007D007C4090011E
:1016B30056E0F8A3E0F9A3E0FAA3E0FB1218A4C0F4
:1016C30004C005C006C0077F007E007D007C4090FB
:1016D300014EE0F8A3E0F9A3E0FAA3E0FB1218A49B
:1016E300A804A905AA06AB07D007D006D005D004E5
:1016F3001217B312525E7B247A0B7998783A121838
:10170300A4A804A905AA06AB07D007D006D005D024
:10171300041217AFC004C005C006C0077F007E00D7
:101723007D007C4090014EE0F8A3E0F9A3E0FAA32A
:10173300E0FB1218A490015AE0F8A3E0F9A3E0FA41
:10174300A3E0FB1217AF12525E7BE07A2D799078FB
:101753003A1218A4A804A905AA06AB07D007D00615
:10176300D005D0041217AF900166121F5E9001627C
:10177300E0FCA3E0FDA3E0FEA3E0FF90015EE0F840
:10178300A3E0F9A3E0FAA3E0FB1217B3900166E02C
:10179300F8A3E0F9A3E0FAA3E0FB1217B37B487ABE
:0817A3005179C778451218A422
:0117AB00221B
:0B29D500900108EBF0A3EAF0A3E9F08A
:1029E00090010EE0FCA3E0FDA3E0FEA3E0FFEC12EB
:1029F0001AC87B007A81798878C61217B3900112C1
:102A0000E0F8A3E0F9A3E0FAA3E0FB1217B390010A
:102A100016121F5E7F0A7EEB7D157C3D900116E04D
:102A2000F8A3E0F9A3E0FAA3E0FB1218A47B7F7AF5
:102A30004F7940783F1217B31266E090011A121FC7
:102A40005E7F8C7EA67D147C3D900116E0F8A3E0AD
:102A5000F9A3E0FAA3E0FB1218A47B367A9079522E
:102A6000783F1217B31266E090011E121F5E7F4D71
:102A70007E6C7D337C3B900116E0F8A3E0F9A3E087
:102A8000FAA3E0FB1218A47B857AEA797E783F12DC
:102A900017B31266E0900122121F5E7F217EB47D83
:102AA0000A7C3D900116E0F8A3E0F9A3E0FAA3E068
:102AB000FB1218A47BD37A697979783F1217B31285
:102AC00066E0900126121F5E7F477E857D167C3D65
:102AD000900116E0F8A3E0F9A3E0FAA3E0FB1218D6
:102AE000A47B9F7A027900783D1217B31266E090BA
:102AF000012A121F5E7F007E007D007C409001262F
:102B0000E0F8A3E0F9A3E0FAA3E0FB1218A4125244
:102B1000747BB07A727928783F1218A4C004C0057B
:102B2000C006C00790011EE0FCA3E0FDA3E0FEA3E9
:102B3000E0FF1252747B7D7A3F79C978401218A465
:102B4000A804A905AA06AB07D007D006D005D00473
:102B50001217B3C004C005C006C0077F007E007D09
:102B6000007C40900126E0F8A3E0F9A3E0FAA3E09E
:102B7000FB1218A4A804A905AA06AB0790011EE041
:102B8000FCA3E0FDA3E0FEA3E0FF1217AF12527416
:102B90007B6F7A1279A3783F1218A4A804A905AA1A
:102BA00006AB07D007D006D005D0041217AFC0047B
:102BB000C005C006C007900122E0FCA3E0FDA3E031
:102BC000FEA3E0FF1252747BC97A76793E783E12FA
:102BD00018A4A804A905AA06AB07D007D006D005FB
:102BE000D0041217AF9001CAE0F8A3E0F9A3E0FA0D
:102BF000A3E0FB1218A490011AE0F8A3E0F9A3E007
:102C0000FAA3E0FB1217B390012E121F5E90012E63
:102C1000E0FCA3E0FDA3E0FEA3E0FFC004C005C00C
:102C200006C0077F007E007D007C4090012AE0F80E
:102C3000A3E0F9A3E0FAA3E0FB1218A41252747BFC
:102C4000D57A7879E9783D1218A4C004C005C00689
:102C5000C0077F007E007D007C4090011EE0F8A34D
:102C6000E0F9A3E0FAA3E0FB1218A41252747BD19E
:102C70007A22795B783E1218A4D003D002D001D01A
:102C8000001217AFC004C005C006C0077F007E0059
:102C90007D007C40900126E0F8A3E0F9A3E0FAA3D0
:102CA000E0FB1218A4C004C005C006C0077F007E68
:102CB000007D007C4090011EE0F8A3E0F9A3E0FA5B
:102CC000A3E0FB1218A4D003D002D001D000121749
:102CD000AF1252747BFC7AA97971783D1218A4A8BE
:102CE00004A905AA06AB07D007D006D005D0041268
:102CF00017AFC004C005C006C0077F007E007D007E
:102D00007C40900126E0F8A3E0F9A3E0FAA3E0FB01
:102D10001218A4C004C005C006C007900122E0FC40
:102D2000A3E0FDA3E0FEA3E0FF90011EE0F8A3E016
:102D3000F9A3E0FAA3E0FB1217B3D003D002D0014D
:102D4000D0001217AF1252747BD57A787969783D2A
:102D50001218A4A804A905AA06AB07D007D006D06C
:102D600005D0041217AF9001CAE0F8A3E0F9A3E080
:102D7000FAA3E0FB1218A4A804A905AA06AB07D081
:102D800007D006D005D0041217B390012E121F5E93
:102D90007F007E007D007C40900126E0F8A3E0F9F2
:102DA000A3E0FAA3E0FB1218A41252747BE37AC7E3
:102DB0007928783F1218A4C004C005C006C0079047
:102DC000011EE0FCA3E0FDA3E0FEA3E0FF125274AD
:102DD0007B9E7A5E79C778401218A4A804A905AA38
:102DE00006AB07D007D006D005D0041217B3C00435
:102DF000C005C006C0077F007E007D007C409001BA
:102E000026E0F8A3E0F9A3E0FAA3E0FB1218A4A8D7
:102E100004A905AA06AB0790011EE0FCA3E0FDA3F0
:102E2000E0FEA3E0FF1217AF1252747BE57AD0796F
:102E3000A2783F1218A4A804A905AA06AB07D007D8
:102E4000D006D005D0041217AF9001CAE0F8A3E075
:102E5000F9A3E0FAA3E0FB1218A490012AE0F8A37A
:102E6000E0F9A3E0FAA3E0FB1217B3900132121FBE
:102E70005E7F007E007D007C40900126E0F8A3E0AC
:102E8000F9A3E0FAA3E0FB1218A4A804A905AA0676
:102E9000AB0790012AE0FCA3E0FDA3E0FEA3E0FF66
:102EA0001217AF1252747B067A817915783E121888
:102EB000A4C004C005C006C007900132E0FCA3E036
:102EC000FDA3E0FEA3E0FF1252747BA67A9B79A4D7
:102ED00078401218A4D003D002D001D0001217AF4E
:102EE0009001CAE0F8A3E0F9A3E0FAA3E0FB12180E
:102EF000A4900136121F5E90012EE0FCA3E0FDA31A
:102F0000E0FEA3E0FF125274C004C005C006C00773
:102F1000900136E0FCA3E0FDA3E0FEA3E0FF125227
:102F20005EA804A905AA06AB07D007D006D005D035
:102F3000041218A47B327AAF79CB783E1218A4C061
:102F400004C005C006C007900136E0FCA3E0FDA365
:102F5000E0FEA3E0FF1252747BDB7ADE796A783FF1
:102F60001218A4A804A905AA06AB07D007D006D05A
:102F700005D0041217B390010BE0FBA3E0FAA3E025
:102F8000F9121EEC90010BE0FBA3E0FAA3E0F912AA
:102F90001ECC90010BE0FBA3E0FAA3E0F9121F3E68
:102FA0001218A4A804A905AA06AB077F007E007D1D
:102FB000807C3F1217AF1260E79000D0121F5E9026
:102FC000010BE0FBA3E0FAA3E0F9121ECC12637937
:102FD00090010BE0FBA3E0FAA3E0F9121EEC9001D4
:102FE0002EE0FCA3E0FDA3E0FEA3E0FF12525EC0D2
:102FF00004C005C006C007900136E0FCA3E0FDA3B5
:10300000E0FEA3E0FF12525EA804A905AA06AB07E2
:10301000D007D006D005D0041218A4C004C005C043
:1030200006C00790010BE0FBA3E0FAA3E0F9121E33
:10303000CC12525EA804A905AA06AB07D007D00699
:10304000D005D0041219AD90013A121F5E90012EE6
:10305000E0FCA3E0FDA3E0FEA3E0FF125274C00475
:10306000C005C006C007900136E0FCA3E0FDA3E068
:10307000FEA3E0FF12525EA804A905AA06AB07D082
:1030800007D006D005D0041218A47BDB7ADE796A5B
:10309000783F1218A4C004C005C006C007900136CE
:1030A000E0FCA3E0FDA3E0FEA3E0FF1252747B323C
:1030B0007AAF79CB783E1218A4A804A905AA06AB6A
:1030C00007D007D006D005D0041217AFC004C00542
:1030D000C006C00790010BE0FBA3E0FAA3E0F912E1
:1030E0001ECC12525EA804A905AA06AB07D007D0D1
:1030F00006D005D0041219AD90013E121F5E90015A
:103100003EE0FCA3E0FDA3E0FEA3E0FFC004C00599
:10311000C006C00790013AE0FCA3E0FDA3E0FEA3D7
:10312000E0FF9000D0121F5ED007D006D005D0047B
:10313000126379900108E0FBA3E0FAA3E0F9121E04
:10314000EC900108E0FBA3E0FAA3E0F9121ECC7BAF
:10315000007A0079007800121A4A6030402E9001FF
:1031600008E0FBA3E0FAA3E0F9C003C002C001122B
:103170001ECC9001CEE0F8A3E0F9A3E0FAA3E0FBB7
:103180001217B3D001D002D003121EEC900108E058
:10319000FBA3E0FAA3E0F9121ECC9001CEE0F8A365
:1031A000E0F9A3E0FAA3E0FB121A4A502E900108BE
:1031B000E0FBA3E0FAA3E0F9C003C002C001121EC5
:1031C000CC9001CEE0F8A3E0F9A3E0FAA3E0FB1273
:0B31D00017AFD001D002D003121EEC9C
:0131DB0022D1
:0B3FC100900190EBF0A3EAF0A3E9F000
:103FCC00900196E0FCA3E0FDA3E0FEA3E0FFEC1261
:103FDC001AC87B007A81798878C61217B390019A37
:103FEC00E0F8A3E0F9A3E0FAA3E0FB1217B37B001F
:103FFC007AAD790E78471219AD90019E121F5E7F33
:10400C00A67EFE7DC77C4290019EE0F8A3E0F9A35A
:10401C00E0FAA3E0FB1218A47B917AEA797E783F50
:10402C001217B31266E09001A2121F5E7F117E235D
:10403C007D5F7C3790019EE0F8A3E0F9A3E0FAA342
:10404C00E0FB1218A4A804A905AA06AB077F507EB2
:10405C00AC7DAE7C3B1217AF1266E0C004C005C04D
:10406C0006C0079001A2E0FCA3E0FDA3E0FEA3E0E4
:10407C00FF125274A804A905AA06AB07D007D006F4
:10408C00D005D0041218A4C004C005C006C0077F18
:10409C00187E017DC87C4290019EE0F8A3E0F9A354
:1040AC00E0FAA3E0FB1218A47B327AE47946783F5D
:1040BC001217B31266E0A804A905AA06AB07D0072D
:1040CC00D006D005D0041217B3C004C005C006C07A
:1040DC00077F007E007D007C409001A2E0F8A3E009
:1040EC00F9A3E0FAA3E0FB1218A41252747B0C7A29
:1040FC0034796978381218A4A804A905AA06AB0764
:10410C00D007D006D005D0041217B39001A6121F09
:10411C005E7F147E6A7D177C3890019EE0F8A3E0E8
:10412C00F9A3E0FAA3E0FB1218A4A804A905AA06B7
:10413C00AB077F6D7E6A7D857C3D1217AF1266E002
:10414C009001AA121F5E9001A6E0FCA3E0FDA3E083
:10415C00FEA3E0FF1252B0C004C005C006C0079019
:10416C0001AAE0FCA3E0FDA3E0FEA3E0FF12525E77
:10417C00A804A905AA06AB07D007D006D005D00421
:10418C001218A4125540900190E0FBA3E0FAA3E0B2
:10419C00F9121EEC9001CEE0F8A3E0F9A3E0FAA32B
:1041AC00E0FB9001A6E0FCA3E0FDA3E0FEA3E0FF92
:1041BC001219AD125A649001CEE0F8A3E0F9A3E015
:1041CC00FAA3E0FB1218A4A804A905AA06AB079051
:1041DC0001A6E0FCA3E0FDA3E0FEA3E0FF1217AFF5
:1041EC009001AE121F5E7F007E007DC07C3F90016F
:1041FC00D2E0F8A3E0F9A3E0FAA3E0FB1218A49034
:10420C0001AEE0F8A3E0F9A3E0FAA3E0FB121A4A2E
:10421C00505A7F007E007D007C3F9001D2E0F8A3D5
:10422C00E0F9A3E0FAA3E0FB1218A49001AEE0F8C9
:10423C00A3E0F9A3E0FAA3E0FB121A4A402E900186
:10424C0090E0FBA3E0FAA3E0F9C003C002C00112A6
:10425C001ECC9001D2E0F8A3E0F9A3E0FAA3E0FBB6
:10426C001217B3D001D002D003121EEC900190E0D3
:10427C00FBA3E0FAA3E0F9C003C002C001121ECCFC
:10428C00C004C005C006C007900190E0FBA3E0FA93
:10429C00A3E0F9121ECC9001CEE0F8A3E0F9A3E064
:1042AC00FAA3E0FB1219AD125A649001CEE0F8A308
:1042BC00E0F9A3E0FAA3E0FB1218A4A804A905AA4C
:1042CC0006AB07D007D006D005D0041217AFD0012B
:1042DC00D002D003121EEC9001A6E0FCA3E0FDA3DB
:1042EC00E0FEA3E0FF125274C004C005C006C00774
:1042FC009001AAE0FCA3E0FDA3E0FEA3E0FF1252B4
:10430C0074A804A905AA06AB07D007D006D005D01F
:10431C00041218A4900193E0FBA3E0FAA3E0F912B5
:10432C001EEC900193E0FBA3E0FAA3E0F9121ECC83
:10433C00900193E0FBA3E0FAA3E0F9121F3E1218E0
:10434C00A4A804A905AA06AB077F007E007D807C8B
:10435C003F1217AF1260E79000D0121F5E900193CE
:10436C00E0FBA3E0FAA3E0F9121ECC1263799001F2
:0C437C0093E0FBA3E0FAA3E0F9121EECB2
:014388002212
:0B31DC0090016AEBF0A3EAF0A3E9F019
:1031E7007F927E0A7D867C3E900170E0F8A3E0F92D
:1031F700A3E0FAA3E0FB1218A4900174E0F8A3E09F
:10320700F9A3E0FAA3E0FB1217AF90017C121F5E4F
:103217007F007E007D007C0090017CE0F8A3E0F950
:10322700A3E0FAA3E0FB121A4A502790017CE0FCC6
:10323700A3E0FDA3E0FEA3E0FF9001CEE0F8A3E04A
:10324700F9A3E0FAA3E0FB1217B390017C121F5E0B
:1032570080489001CEE0FCA3E0FDA3E0FEA3E0FFE1
:1032670090017CE0F8A3E0F9A3E0FAA3E0FB121ACF
:103277004A6027402590017CE0FCA3E0FDA3E0FE27
:10328700A3E0FF9001CEE0F8A3E0F9A3E0FAA3E002
:10329700FB1217AF90017C121F5E90017CE0F8A330
:1032A700E0F9A3E0FAA3E0FB90001EE0FCA3E0FD39
:1032B700A3E0FEA3E0FF1217AF900016121F5E9067
:1032C7000016E0FCA3E0FDA3E0FEA3E0FF12525EC0
:1032D700C004C005C006C00790001AE0FCA3E0FDCB
:1032E700A3E0FEA3E0FF12525EA804A905AA06AB5D
:1032F70007D007D006D005D0041218A4C004C00513
:10330700C006C007900178E0FCA3E0FDA3E0FEA3A0
:10331700E0FF12525EA804A905AA06AB07D007D0A2
:1033270006D005D0041218A4C004C005C006C00703
:1033370090001AE0FCA3E0FDA3E0FEA3E0FF125219
:1033470074C004C005C006C007900178E0FCA3E084
:10335700FDA3E0FEA3E0FF125274A804A905AA0684
:10336700AB07D007D006D005D0041218A4A804A92B
:1033770005AA06AB07D007D006D005D0041217B3AD
:10338700900180121F5E900180E0FCA3E0FDA3E0A6
:10339700FEA3E0FF900180E0F8A3E0F9A3E0FAA321
:1033A700E0FB1218A4A804A905AA06AB077F007EB4
:1033B700007D807C3F1217AF1260E7900184121FD7
:1033C7005E900180E0FCA3E0FDA3E0FEA3E0FFC068
:1033D70004C005C006C007900184E0FCA3E0FDA37C
:1033E700E0FEA3E0FF9000D0121F5ED007D006D00A
:1033F70005D00412637990016DE0FBA3E0FAA3E026
:10340700F9121EEC90016DE0FBA3E0FAA3E0F912BC
:103417001ECC12525EC004C005C006C00790016DE5
:10342700E0FBA3E0FAA3E0F9121ECC125274D0031A
:10343700D002D001D0001219ADC004C005C006C02B
:103447000790001AE0FCA3E0FDA3E0FEA3E0FF1253
:10345700525EC004C005C006C00790001AE0FCA376
:10346700E0FDA3E0FEA3E0FF125274D003D002D028
:1034770001D0001219ADA804A905AA06AB07D00709
:10348700D006D005D0041218A4C004C005C006C0D9
:103497000790016DE0FBA3E0FAA3E0F9121ECC123E
:1034A700525EC004C005C006C00790001AE0FCA326
:1034B700E0FDA3E0FEA3E0FF12525EA804A905AA5F
:1034C70006AB07D007D006D005D0041218A4C00455
:1034D700C005C006C007900178E0FCA3E0FDA3E0AB
:1034E700FEA3E0FF125274D003D002D001D0001225
:1034F70019ADD003D002D001D0001217AF90018CC4
:10350700121F5E900178E0FCA3E0FDA3E0FEA3E0BC
:10351700FF12525EC004C005C006C00790001AE043
:10352700FCA3E0FDA3E0FEA3E0FF12525EA804A9FE
:1035370005AA06AB07D007D006D005D0041218A4F9
:10354700C004C005C006C007900016E0FCA3E0FD5C
:10355700A3E0FEA3E0FF12525EA804A905AA06ABEA
:1035670007D007D006D005D0041218A4C004C005A0
:10357700C006C007900178E0FCA3E0FDA3E0FEA32E
:10358700E0FF125274C004C005C006C00790001ABD
:10359700E0FCA3E0FDA3E0FEA3E0FF125274A80441
:1035A700A905AA06AB07D007D006D005D004121884
:1035B700A4A804A905AA06AB07D007D006D005D052
:1035C700041217B3900188121F5E900178E0FCA3E4
:1035D700E0FDA3E0FEA3E0FF12525EC004C005C0F9
:1035E70006C007900016E0FCA3E0FDA3E0FEA3E001
:1035F700FF125274A804A905AA06AB07D007D00684
:10360700D005D0041218A4C004C005C006C0079096
:103617000188E0FCA3E0FDA3E0FEA3E0FF900188A2
:10362700E0F8A3E0F9A3E0FAA3E0FB1218A4A804CA
:10363700A905AA06AB077F007E007D807C3F121795
:10364700AF1260E7A804A905AA06AB07D007D00602
:10365700D005D0041219AD900188121F5E90018821
:10366700E0FCA3E0FDA3E0FEA3E0FFC004C005C0AB
:1036770006C00790018CE0FCA3E0FDA3E0FEA3E0F9
:10368700FF9000D0121F5ED007D006D005D00412DD
:10369700637990016AE0FBA3E0FAA3E0F9121EEC5C
:1036A70090016AE0FBA3E0FAA3E0F9121ECC7B00CD
:1036B7007A0079007800121A4A6030402E90016A29
:1036C700E0FBA3E0FAA3E0F9C003C002C001121EA9
:1036D700CC9001CEE0F8A3E0F9A3E0FAA3E0FB1257
:0B36E70017B3D001D002D003121EEC7C
:0136F20022B5
:10603700323B171C0205006400640001000007A33F
:106047000087038400640708038406820569000744
:1060570000020009003B003B0017001C000C006316
:1060670000C700C70002000A0E0F03840E0F038447
:106077000E0F07080E0F070800070005000E0000A7
:106087000000000000010001000000010001000005
:1060970000000000000000000000000000000000F9
:1060A70000000000000000000000000300000003E3
:1060B70000020003000200030003000200030002C5
:1060C70000030000000300010003000200030002B8
:0C60D700000300030002000300020003AD
:06673700C112C114C113E0
:1065B9009000107432F0900011743BF09000127446
:1065C90017F0900013741CF09000147402F09000FE
:1065D900157405F0124C33755D00755E00D3E55EE8
:1065E900940EE55D64809480503CE55E25E0FFE50E
:1065F9005D33FE743D2FF58274603EF583E493FCB0
:10660900740193FDE55E25E0FFE55D33FE74222FFD
:10661900F58274003EF583ECF0A3EDF0055EE55ECE
:0A6629007002055D80B7124D3722A4
:103B760090003FE0F558D3E55864809482400BC32B
:103B8600E558648094865002C212E5A064FFFFEFF8
:103B96005407F55AE55A6006C29CC2988002D29C28
:103BA600E55A5406FFEF6027055CE55CD3940A40AE
:103BB6000F75590AC3E558648094865003755C0AEC
:103BC600E55CD39414400E755964755C14800675D3
:103BD6005C00755901AF58EF3395E0FEEF25E0FF25
:103BE600EE33FE74852FF58274603EF583E493F51B
:103BF60056740193F557AF58EF3395E0FEEF25E085
:103C0600FFEE33FE745B2FF58274603EF583E4931A
:103C1600F554740193F555E5586403706B900015DF
:103C2600E0FFEF75F004121D86AFF0EF602E9000F6
:103C360014E0FFEF3395E0FEEF25E0FFEE33FE7470
:103C4600AF2FF58274603EF583E493FE740193FF13
:103C5600EF2555F555EE3554F554802C900014E0BB
:103C6600FFEF3395E0FEEF25E0FFEE33FE74C92F3C
:103C7600F58274603EF583E493FE740193FFEF25AD
:103C860055F555EE3554F554E55AB4011090002813
:103C9600E0FEA3E0FFEF4E7004055B8003755B005A
:103CA600E55BC394144008755B00A212B39212D36D
:103CB600E55A648094815003023F65C3E5586480E9
:103CC60094864003023D8B124C88E55A6404705575
:103CD600AF58EF3395E0FE74102FF58274003EF571
:103CE60083E02559F0AF58EF3395E0FE74102FF5B9
:103CF6008274003EF583E0FFEF3395E0FED3EF9547
:103D060055E5546480F8EE6480984016AF57AE5877
:103D1600EEFD3395E0FC74102DF58274003CF583BE
:103D2600EFF0124C33E55A6402705AAF58EF3395F0
:103D3600E0FE74102FF58274003EF583E0FFC3EFBA
:103D46009559FFEFF0AF58EF3395E0FE74102FF55D
:103D56008274003EF583E0FFEF3395E0FEC3EF95F6
:103D660057E5566480F8EE6480985016AF55AE5805
:103D7600EEFD3395E0FC74102DF58274003CF5835E
:103D8600EFF0124C33C3E558648094865003023E2C
:103D9600A774FA2558F558E55A64047072AF59EFBE
:103DA600FD7C00AF58EF3395E0FEEF25E0FFEE33E4
:103DB600FE74222FF58274003EF583EC8DF0121E00
:103DC60048AF58EF3395E0FEEF25E0FFEE33FE7483
:103DD600222FF58274003EF583E0FEA3E0FFD3EFC9
:103DE6009555E5546480F8EE648098401FAF58EF0F
:103DF6003395E0FEEF25E0FFEE33FE74222FF582C9
:103E060074003EF583E556F0A3E557F0124D37E50D
:103E16005A64026003023EA1AF58EF3395E0FEEF0D
:103E260025E0FFEE33FE74222FF58274003EF58303
:103E3600C083C082E0FEA3E0FFAD597C00C3EF9DC6
:103E4600FFEE9CFED082D083EEF0A3EFF0AF58EFEA
:103E56003395E0FEEF25E0FFEE33FE74222FF58268
:103E660074003EF583E0FEA3E0FFC3EF9557E556E9
:103E76006480F8EE648098501FAF58EF3395E0FEEB
:103E8600EF25E0FFEE33FE74222FF58274003EF537
:103E960083E554F0A3E555F0124D3774062558F521
:103EA60058900028E0FEA3E0FFEF4E705CE55AB4A0
:103EB60005263014230558AF58D3EF6480949340F9
:103EC60003755800C214AF58EF3395E0FE90003EDC
:103ED600EEF0A3EFF0124D37E55A64036003023F9C
:103EE6006530147B1558AF58C3EF64809480500337
:103EF600755813C214AF58EF3395E0FE90003EEEAE
:103F0600F0A3EFF0124D378056E55AB4052630146B
:103F1600230558AF58D3EF64809492400375580038
:103F2600C214AF58EF3395E0FE90003EEEF0A3EFDB
:103F3600F0124D37E55AB403263014231558AF58FE
:103F4600C3EF648094805003755812C214AF58EFC3
:103F56003395E0FE90003EEEF0A3EFF0124D37E50C
:103F66005AB40102D214E55A5406FFEF60109000CD
:103F76003EE0FEA3E0FFEF64094E7002C217900117
:103F8600DFE0FEA3E0FF900028E0FCA3E0FDED6F7C
:103F96007002EC6E6002C217900028E0FEA3E0FFFC
:103FA6009001DFEEF0A3EFF030A302D21320A30AB4
:0A3FB600301307C213A217B39217CD
:013FC00022DE
:104C3300124D8074A0124D987402124D989000107A
:104C43007C03E0124D59124D98A3DCF6E0124D5946
:104C5300F5F0A3A3E0030354C045F0124D98900070
:104C630014E0124D59124D98C2B4124D73124D8077
:104C730074A0124D9874F0124D98A3E0124D98C28F
:104C8300B4124D7322124D8074A0124D9874021207
:104C93004D98124D8074A004124D98900010124D3F
:104CA300BD124D61F0A3124DD0124DBD124D61F0F6
:104CB300A3124DD0124DBD124D61F0A3124DD0126F
:104CC3004DBDFB543F124D61F0A3124DD0124DBDAB
:104CD300FA541F124D61F0EB23235403FD124DCA06
:104CE300C2B4124D73124D8074A0124D9874F01219
:104CF3004D98124D8074A004124D98124DBDFB5473
:104D030003C39D2405838007030201000302012BD3
:104D1300A3F0F5F0124DCAC2B4124D73124D807454
:104D2300A0124D9874F0124D98E5F0124D98C2B44C
:104D3300124D73227AA07B807C1E900022124E10AB
:104D4300227AA07B80124DD8ED900022F07AA0A3A6
:104D53007C1D124E452275F00A84C425F022C0E062
:0D4D6300C4540F75F00AA4F5F0D0E0540F11
:104D700025F02200D2B5000000D2B40000000022CD
:104D8000124D73C2B4000000C2B500000022D2B5BB
:104D9000000000C2B50000227E083392B4124D8E8E
:104DA000DEF833D2B40000A2B450040000A2B41262
:104DB0004D8E400122C2B40000124D73227E08A223
:104DC000B43300124D8EDEF7C322D2B4124D8E22C0
:104DD000C2B4124D8ED2B422124D80EA124D98EB1D
:104DE000124D98124D80EA04124D98124DBDFD12DD
:104DF0004DCAC2B4124D7322124D80EA124D98EB87
:104E0000124D98E6124D9808DCF9C2B4124D732287
:104E1000124D80EA124D98EB124D98E0124D98A376
:104E2000DCF9C2B4124D7322124D80EA04124D987F
:104E30008003124DD0124DBDF608DCF6124DCAC2E9
:104E4000B4124D7322124D80EA04124D9880031261
:104E50004DD0124DBDF0A3DCF6124DCAC2B4124DB6
:024E60007322BB
:10496A00202020202531642E253032642025303243
:10497A0062753A25303262753A25303262752020E6
:10498A00202000202020202532642E253164202575
:10499A00303262753A25303262753A2530326275A4
:1049AA002020202000253033642E25316420202544
:1049BA003032642E25316420415A2F454C31202053
:1049CA002000253033642E253164202025303264BE
:1049DA002E25316420415A2F454C322020200025B3
:1049EA003033642E2531642020253032642E25315F
:1049FA00642052412F44454320202000253033644F
:104A0A002E2531645720253032642E2531644E20FC
:104A1A004C4F2F4C41202020002530326275202037
:104A2A00202530326275202025303262753A2530D1
:104A3A003262753A253032627520202020002530F6
:104A4A00352E31662020253032642E25316420200F
:104A5A00202020202025303264202000202B2530E1
:104A6A0031642E2530316420202B253031642E25E7
:104A7A0030316420434F52202053545020002530B7
:104A8A0033642E2531642020253032642E2531648A
:104A9A0020414E5420202531642E253164200020E7
:104AAA002020204F20452035204A2046204C202017
:104ABA00202020002020202020202020454D452095
:104ACA0020202020202020200020416E74656E6E58
:104ADA006120436F6E74726F6C6C657220002020C7
:104AEA0020202020207620312E3020202020202037
:104AFA002020002020204A414E4645424D41524145
:104B0A0050524D41594A554E4A554C4155475345C5
:104B1A00504F43544E4F56444543004D4F4F4E203D
:104B2A002053554E20202043415353494F43594760
:104B3A004E55535341474954545441555255534C79
:104B4A00454F20202041515541522E52412F444574
:104B5A0043415A2F454C32415A2F454C3100326D50
:104B6A003A37303A32333A31333A36636D31304775
:104B7A000020535349203130626974283732302972
:104B8A002020202020205353493131626974283172
:104B9A0038303029202020202020535349313262D6
:104BAA00697428333630302920202020202053539E
:104BBA00495F6772617928343039362920202020EC
:104BCA00202041322D532D53203132206269742026
:104BDA0020202020204D414232355F3130626974F5
:104BEA003130323420202020204D414232355F318D
:104BFA00316269743230343820202020204D4142FD
:104C0A0032355F31326269743430393620202020DF
:104C1A0020000F0C09010306171D664C030903093E
:094C2A000309030956010102040B
:10002E00E55A64016003125708200D0302060CC244
:10003E000D30120C900028E0FEA3E0FFEF4E601191
:10004E0090003EE0FEA3E0FFEF64134E600302015A
:10005E00E390003CE0FEA3E0FFC3EF9404EE648067
:10006E00948040030200FCAF1CAE1B12000EEF2466
:10007E0005FFEE3400FE7C007D0A121E128E638F89
:10008E00647B017A00796CC003C002C0017BFF7AE9
:10009E0049796A9000DBEBF0A3EAF0A3E9F0AE63D6
:1000AE00AF647C007D64121E129000DEEEF0A3EFB2
:1000BE00F0AE63AF647C007D64121E129000E0EC23
:1000CE00F0A3EDF0900012E0FF9000E2EFF0900050
:1000DE0011E0FF9000E3EFF0900010E0FF9000E4DD
:1000EE00EFF0D001D002D003123758020180AF1CBE
:1000FE00AE1B12000EEF2432FFEE3400FE7C007DAC
:10010E0064121E128E638F647B017A00796CC003B9
:10011E00C002C0017BFF7A49798D9000DBEBF0A322
:10012E00EAF0A3E9F0AE63AF647C007D0A121E1202
:10013E009000DEEEF0A3EFF0AE63AF647C007D0ABC
:10014E00121E129000E0ECF0A3EDF0900012E0FF12
:10015E009000E2EFF0900011E0FF9000E3EFF090DE
:10016E000010E0FF9000E4EFF0D001D002D00312B7
:10017E003758751500D3E515648094825042AF153B
:10018E0090003DE0FE75F003EEA4F58285F083E568
:10019E00822FF582E43583F583E5822468F582E5C6
:1001AE0083344BF583E493FFAE15EEFD3395E0FCFF
:1001BE00746C2DF58274003CF583EFF0051580B557
:1001CE00C3E51B64809480400302059C90006F740D
:1001DE002DF002059C90003EE0FEA3E0FFEF640AC6
:1001EE004E601190003EE0FEA3E0FFEF640B4E6008
:1001FE00030202877B017A00796CC003C002C00142
:10020E007BFF7A4979AF9000DBEBF0A3EAF0A3E92C
:10021E00F090002AE0FEA3E0FF7C007D0A121E1281
:10022E009000DEEEF0A3EFF090002AE0FEA3E0FFD8
:10023E007C007D0A121E129000E0ECF0A3EDF0900F
:10024E00002CE0FEA3E0FF7C007D0A121E1290003F
:10025E00E2EEF0A3EFF090002CE0FEA3E0FF7C00B6
:10026E007D0A121E129000E4ECF0A3EDF0D001D046
:10027E0002D00312375802059C90003EE0FEA3E028
:10028E00FFEF640C4E601190003EE0FEA3E0FFEF26
:10029E00640D4E600302032B7B017A00796CC00360
:1002AE00C002C0017BFF7A4979CC9000DBEBF0A352
:1002BE00EAF0A3E9F090002EE0FEA3E0FF7C007DC3
:1002CE000A121E129000DEEEF0A3EFF090002EE068
:1002DE00FEA3E0FF7C007D0A121E129000E0ECF0FF
:1002EE00A3EDF0900030E0FEA3E0FF7C007D0A124B
:1002FE001E129000E2EEF0A3EFF0900030E0FEA3AD
:10030E00E0FF7C007D0A121E129000E4ECF0A3EDDB
:10031E00F0D001D002D00312375802059C90003E57
:10032E00E0FEA3E0FFEF640E4E601190003EE0FE93
:10033E00A3E0FFEF640F4E60030203F9900034E078
:10034E00FEA3E0FFEF247CF560EE34FCF55FAF60BA
:10035E00AE5F12000E7C007D0A121E12C006C00790
:10036E00AF60AE5F12000E7C007D0A121E1290006E
:10037E00E4ECF0A3EDF0D007D0069000E2EEF0A38F
:10038E00EFF07B017A00796CC003C002C0017BFFE5
:10039E007A4979E99000DBEBF0A3EAF0A3E9F0905B
:1003AE000032E0FEA3E0FF7C007D0A121E129000D8
:1003BE00DEEEF0A3EFF0900032E0FEA3E0FF7C0053
:1003CE007D0A121E129000E0ECF0A3EDF0D001D0E9
:1003DE0002D003123758C3E55F6480948040030255
:1003EE00059C900072742DF002059C90003EE0FE7C
:1003FE00A3E0FFEF64104E601190003EE0FEA3E01C
:10040E00FFEF64114E60030204F6900036E0FEA387
:10041E00E0FFEF24F8F562EE34F8F561900038E075
:10042E00FEA3E0FFEF247CF560EE34FCF55FAF62D7
:10043E00AE6112000E7C007D0A121E12C006C007AD
:10044E00AF62AE6112000E7C007D0A121E12C00455
:10045E00C005AF60AE5F12000E7C007D0A121E1248
:10046E00C006C007AF60AE5F12000E7C007D0A12A0
:10047E001E129000E4ECF0A3EDF0D007D006900031
:10048E00E2EEF0A3EFF0D005D0049000E0ECF0A384
:10049E00EDF0D007D0069000DEEEF0A3EFF07B017A
:1004AE007A00796CC003C002C0017BFF7A4A7906DC
:1004BE009000DBEBF0A3EAF0A3E9F0D001D002D07C
:1004CE0003123758C3E56164809480500690007122
:1004DE007445F0C3E55F64809480400302059C90F0
:1004EE0000767453F002059C7B017A00796CC00390
:1004FE00C002C0017BFF7A4A79239000DBEBF0A3A8
:10050E00EAF0A3E9F0900013E0FF9000DEEFF09028
:10051E000015E0FF9000DFEFF0900012E0FF90007A
:10052E00E0EFF0900011E0FF9000E1EFF09000108E
:10053E00E0FF9000E2EFF0D001D002D00312375866
:10054E00751500D3E515648094825042AF15900066
:10055E0014E0FE75F003EEA4F58285F083E5822F9C
:10056E00F582E43583F583E58224FDF582E5833457
:10057E004AF583E493FFAE15EEFD3395E0FC746E01
:10058E002DF58274003CF583EFF0051580B59000D3
:10059E0028E0FEA3E0FFC3EF9402EE648094805047
:1005AE003290003EE0FEA3E0FFC3EF940AEE6480BB
:1005BE009480401390003EE0FEA3E0FFD3EF941131
:1005CE00EE64809480400C90007E7444F090007F26
:1005DE007445F07F0012571A751500D3E515648027
:1005EE009493501AAF15EF3395E0FE746C2FF5828D
:1005FE0074003EF583E0FF1256E1051580DD200EF6
:10060E000302080CC20E90003EE0FEA3E0FFC3EF13
:10061E00940AEE64809480401590003EE0FEA3E0C4
:10062E00FFD3EF9411EE648094805002C2129001B9
:10063E00CAE0F8A3E0F9A3E0FAA3E0FB900004E01F
:10064E00FCA3E0FDA3E0FEA3E0FF1219AD12683596
:10065E007B007A00792078411218A47B007A007909
:10066E0000783F1217B3121B068E5F8F609001CA7F
:10067E00E0F8A3E0F9A3E0FAA3E0FB900068E0FC49
:10068E00A3E0FDA3E0FEA3E0FF1219AD1268357BD7
:10069E00007A007900783F1217B3121B068E658F11
:1006AE00667B017A007984C003C002C0017BFF7AA9
:1006BE004A79489000DBEBF0A3EAF0A3E9F0900151
:1006CE00CAE0F8A3E0F9A3E0FAA3E0FB90000CE087
:1006DE00FCA3E0FDA3E0FEA3E0FF1219AD9000DE47
:1006EE00121F5EAE5FAF607C007D0A121E1290007C
:1006FE00E2EEF0A3EFF0AE5FAF607C007D0A121E5B
:10070E00129000E4ECF0A3EDF09000E6E565F0A3A6
:10071E00E566F0D001D002D0031237587F007E007C
:10072E007D007C00900004E0F8A3E0F9A3E0FAA3BA
:10073E00E0FB121A4A500690008A742DF0751500CF
:10074E00D3E515648094855042AF15900029E0FEE4
:10075E0075F006EEA4F58285F083E5822FF582E42E
:10076E003583F583E5822425F582E583344BF583C5
:10077E00E493FFAE15EEFD3395E0FC74902DF582FB
:10078E0074003CF583EFF0051580B5900028E0FE6F
:10079E00A3E0FFC3EF9402EE64809480400E9000BD
:1007AE00967420F09000977420F080217F007E00D8
:1007BE007D007C00900068E0F8A3E0F9A3E0FAA3C6
:1007CE00E0FB121A4A5006900095742DF0E55A641B
:1007DE0001602B7F4012571A751500D3E515648002
:1007EE009493501AAF15EF3395E0FE74842FF58273
:1007FE0074003EF583E0FF1256E1051580DD200FF3
:10080E0003020917C20F900022E0FEA3E0FFEF24BF
:10081E009CFFEE34FFFE12000E8E618F629000245C
:10082E00E0FEA3E0FFEF249CFFEE34FFFE12000E6D
:10083E008E5F8F607B017A00799CC003C002C0017D
:10084E007BFF7A4A79669000DBEBF0A3EAF0A3E92E
:10085E00F0AE61AF627C007D0A121E129000DEEED9
:10086E00F0A3EFF0AE61AF627C007D0A121E129013
:10087E0000E0ECF0A3EDF0AE5FAF607C007D0A12FD
:10088E001E129000E2EEF0A3EFF0AE5FAF607C00C0
:10089E007D0A121E129000E4ECF0A3EDF0D001D010
:1008AE0002D003123758900022E0FEA3E0FFC3EF00
:1008BE009464EE64809480500690009D742DF090A8
:1008CE000024E0FEA3E0FFC3EF9464EE6480948006
:1008DE0050069000A3742DF0E55A6401602B7F142E
:1008EE0012571A751500D3E51564809493501AAFFC
:1008FE0015EF3395E0FE749C2FF58274003EF58360
:10090E00E0FF1256E1051580DD201003020B19C21F
:10091E0010900027E0FFEF904C3093FFEF3395E0FF
:10092E00FEAC4AAD4B121E008E438F44AF41AE401B
:10093E0012000E7C007D0A121E12C006C007AF41C7
:10094E00AE4012000E7C007D0A121E129000E4ECE6
:10095E00F0A3EDF0D007D0069000E2EEF0A3EFF09A
:10096E007B017A0079B4C003C002C0017BFF7A4AD2
:10097E0079889000DBEBF0A3EAF0A3E9F0AE45AF87
:10098E00467C007D0A121E129000DEEEF0A3EFF000
:10099E00AE45AF467C007D0A121E129000E0ECF0D0
:1009AE00A3EDF0AE43AF447C007D0A121E12900000
:1009BE00E6EEF0A3EFF0AE43AF447C007D0A121ECC
:1009CE00129000E8ECF0A3EDF0D001D002D00312AB
:1009DE003758C3E5406480948050069000BA742D59
:1009EE00F0A218B39218E508540CFFEFB4080820D3
:1009FE0018059000C4E4F0E508540CFFEFB40409A8
:100A0E002018069000C47401F0E508540CFFEFB4F2
:100A1E000C093017069000C4742AF0E5085403FF41
:100A2E00EFB402093018069000C37402F0E50854C2
:100A3E0003FFEFB401093018069000C37403F0E50C
:100A4E00085403FFEFB403093017069000C3742A4D
:100A5E00F090003EE0FEA3E0FFEF64124E60030252
:100A6E000AEE751500D3E515648094935042AF15C8
:100A7E0090003BE0FE75F014EEA4F58285F083E560
:100A8E00822FF582E43583F583E582247BF582E5BA
:100A9E0083344BF583E493FFAE15EEFD3395E0FC06
:100AAE0074B42DF58274003CF583EFF0051580B516
:100ABE00AE43AF447C007D0A121E12EF2430FF902D
:100ACE0000C5EFF09000C6742EF0AE43AF447C002C
:100ADE007D0A121E12AF05EF2430FF9000C7EFF013
:100AEE007F5412571A751500D3E5156480949350F0
:100AFE001AAF15EF3395E0FE74B42FF58274003EF5
:100B0E00F583E0FF1256E1051580DDE55AB40114B8
:100B1E0090003FE0FFEF904C1C93FF12571A1256B5
:100B2E00FF125711301103020C7C7B017A00796C95
:100B3E00C003C002C0017BFF7A4A79A99000DBEBAB
:100B4E00F0A3EAF0A3E9F0D001D002D00312375897
:100B5E007B017A007984C003C002C0017BFF7A4A10
:100B6E0079BE9000DBEBF0A3EAF0A3E9F0D001D060
:100B7E0002D0031237587B017A00799CC003C00261
:100B8E00C0017BFF7A4A79D39000DBEBF0A3EAF049
:100B9E00A3E9F0D001D002D0031237587B017A00BE
:100BAE0079B4C003C002C0017BFF7A4A79E8900095
:100BBE00DBEBF0A3EAF0A3E9F0D001D002D00312F0
:100BCE0037587F0012571A751500D3E515648094B7
:100BDE0093501AAF15EF3395E0FE746C2FF58274B7
:100BEE00003EF583E0FF1256E1051580DD7F4012D1
:100BFE00571A751500D3E51564809493501AAF15E6
:100C0E00EF3395E0FE74842FF58274003EF583E099
:100C1E00FF1256E1051580DD7F1412571A75150067
:100C2E00D3E51564809493501AAF15EF3395E0FE1B
:100C3E00749C2FF58274003EF583E0FF1256E10599
:100C4E001580DD7F5412571A751500D3E515648093
:100C5E009493501AAF15EF3395E0FE74B42FF582CE
:0F0C6E0074003EF583E0FF1256E1051580DD228C
:10673D00014900014700014800014200C117C1167F
:02674D00C11574
:10680200752400D3E524648094A75004052480F302
:016812002263
:10681300752500D3E525648094935004052580F302
:016823002252
:10682400752600D3E5266480949E5004052680F3E3
:016834002241
:105C4300C290126802752C1F752B00E52BD39407A5
:105C53005011E52CC313F52CA2D7929012680205BC
:105C63002B80E8D290126802D2927527037528E838
:105C7300752C00309110E52815287002152714FFA4
:105C8300AE27EF4E70ED126813752B00E52BD394FE
:105C9300075013126802E52CC313F52C309103430C
:105CA3002C80052B80E6126802AF2C7E00EF752A4C
:105CB30000F5297527037528E8752C00309110E548
:105CC3002815287002152714FFAE27EF4E70ED122A
:105CD3006813752B00E52BD394075013126802E564
:105CE3002CC313F52C309103432C80052B80E61233
:105CF3006802AF2C7E00EF252AF52AEE3529F52917
:105D0300C3E529648094805006752900752A00D361
:105D1300E52A940FE5296480948E400675290E7553
:085D23002A0FC292AE29AF2A3B
:015D2B002255
:105D2C00C29412680275321F753100E531D39407A5
:105D3C005011E532C313F532A2D7929412680205C2
:105D4C003180E8D294126802D296752D03752EE834
:105D5C00753200309510E52E152E7002152D14FF9E
:105D6C00AE2DEF4E70ED126813753100E531D39402
:105D7C00075013126802E532C313F5323095034312
:105D8C003280053180E6126802AF327E00EF75304A
:105D9C0000F52F752D03752EE8753200309510E542
:105DAC002E152E7002152D14FFAE2DEF4E70ED1228
:105DBC006813753100E531D394075013126802E56E
:105DCC0032C313F532309503433280053180E6122D
:105DDC006802AF327E00EF2530F530EE352FF52F0F
:105DEC00C3E52F648094805006752F00753000D366
:105DFC00E530940FE52F6480948E4006752F0E7558
:085E0C00300FC296AE2FAF303B
:015E1400226B
:10679B00125C438E458F46125D2CC374089FFF74A9
:1067AB00079EFE12000EC374849FF54174039EF581
:0867BB0040754A00754B0122F4
:10618F00D290D294D291D295755000755100754C22
:10619F0000754D00753300D3E53364809489504901
:1061AF00126824C290C294126824C3E533648094A9
:1061BF00895004D290D294E5512551F551E55035CF
:1061CF0050F550E54D254DF54DE54C354CF54C2032
:1061DF0091080551E55170020550209508054DE5D0
:1061EF004D7002054C053380AEC290C294754A00C3
:1061FF00754B05AE50AF517C007D05121E008E45CC
:10620F008F46C37468954DFF7401954CFE12000EB6
:10621F00C374B49FF54DE49EF54CAE4CAF4D7C006E
:09622F007D05121E008E408F4116
:016238002243
:10623900D290D294D291D295755000755100754C77
:1062490000754D00753400D3E5346480948A504953
:10625900126824C290C294126824C3E534648094FD
:106269008A5004D290D294E5512551F551E5503523
:1062790050F550E54D254DF54DE54C354CF54C2087
:1062890091080551E55170020550209508054DE525
:106299004D7002054C053480AEC290C294754A0017
:1062A900754B02E55125E0F546E55033F545C374D4
:1062B90084954DFF7403954CFE12000EC374C29F62
:1062C900F54D74019EF54CE54D25E0F541E54C335E
:0262D900F5408E
:0162DB0022A0
:10641600D290D294D291D295755000755100754C98
:1064260000754D00753500D3E5356480948B504971
:10643600126824C290C294126824C3E5356480941D
:106446008B5004D290D294E5512551F551E5503543
:1064560050F550E54D254DF54DE54C354CF54C20A8
:1064660091080551E55170020550209508054DE546
:106476004D7002054C053580AEC290C294754A0037
:10648600754B01855045855146C37408954DFF747B
:1064960007954CFE12000EC374849FF54174039E4B
:0264A600F540BF
:0164A80022D1
:10575F00D292D296D291D295755000755100754C58
:10576F0000754D001268249001E7E4F09001E7E026
:10577F00FFD3EF6480948F5044D290D29412682458
:10578F00C290C294126824E5512551F551E5503568
:10579F0050F550E54D254DF54DE54C354CF54C206C
:1057AF0091080551E55170020550209508054DE50A
:1057BF004D7002054C9001E7E004F080AFC290C23B
:1057CF0094C292C296754A00754B05E551AE50785A
:1057DF0006CEC313CE13D8F9F5518E50E54DAE4C0E
:1057EF007806CEC313CE13D8F9F54D8E4CAC50AD11
:1057FF0051E4121ACD7B007A00793478441218A440
:10580F007B007A00798078441219AD121B067C0058
:10581F007D05121E008E458F46C3E4954DFF740221
:10582F00954CFE12000EC3E49FFD74019EFCEC121A
:10583F001ACD7B007A00793478441218A47B007A51
:10584F0000798078441219AD121B067C007D051279
:06585F001E008E408F4187
:015865002220
:10586600D292D296D291D295755000755100754C50
:1058760000754D001268249001E8E4F09001E8E01C
:10588600FFD3EF6480948F5044D290D29412682450
:10589600C290C294126824E5512551F551E5503560
:1058A60050F550E54D254DF54DE54C354CF54C2064
:1058B60091080551E55170020550209508054DE502
:1058C6004D7002054C9001E8E004F080AFC290C232
:1058D60094C292C296754A00754B02E551AE507855
:1058E60005CEC313CE13D8F9F5518E50E54DAE4C07
:1058F6007805CEC313CE13D8F9F54D8E4CAC50AD0A
:1059060051E4121ACD7B007A0079E178441218A48A
:105916007B007A00790078451219AD121B06EF2537
:10592600E0F546EE33F545C3E4954DFF7404954C1A
:10593600FE12000EC3E49FFD74029EFCEC121ACD0B
:105946007B007A0079E178441218A47B007A00790A
:105956000078451219AD121B06EF25E0F541EE332E
:02596600F5400A
:01596800221C
:10596900D292D296D291D295755000755100754C4C
:1059790000754D001268249001E9E4F09001E9E016
:10598900FFD3EF6480948F5044D290D2941268244C
:10599900C290C294126824E5512551F551E550355C
:1059A90050F550E54D254DF54DE54C354CF54C2060
:1059B90091080551E55170020550209508054DE5FE
:1059C9004D7002054C9001E9E004F080AFC290C22D
:1059D90094C292C296754A00754B01E550C4F854B9
:1059E900F0C868F550E551C4540F48F551E54CC469
:1059F900F854F0C868F54CE54DC4540F48F54DAC62
:105A090050AD51E4121ACD7B007A007961784512C4
:105A190018A47B007A00798078451219AD121B060B
:105A29008E458F46C3E4954DFF7408954CFE1200D0
:105A39000EC3E49FFD74049EFCEC121ACD7B007A20
:105A490000796178451218A47B007A00798078453D
:0A5A59001219AD121B068E408F419A
:015A63002220
:105B5400D290D294D291D295755000755100754C63
:105B640000754D00753600D3E5366480948B505330
:105B7400C290C294753700D3E53764809482500490
:105B8400053780F3C3E5366480948B5004D290D2F9
:105B940094E5512551F551E5503550F550E54D2525
:105BA4004DF54DE54C354CF54C2091080551E5512A
:105BB40070020550209508054DE54D7002054C0511
:105BC4003680A4C290C294754A00754B01AF51AEA1
:105BD400501267EA8E508F51AF4DAE4C1267EA8E69
:105BE4004C8F4DAC50AD51E4121ACD7B007A007944
:105BF4006178451218A47B007A00798078451219DF
:105C0400AD121B068E458F46C3E4954DFF7408956F
:105C14004CFE12000EC3E49FFD74049EFCEC121AA9
:105C2400CD7B007A00796178451218A47B007A0054
:0E5C3400798078451219AD121B068E408F4103
:015C4200223F
:1046890075080F900022E0FEA3E0FFE5532FFFE538
:10469900523EFEEF249CFFEE34FFFEC3EF9546F534
:1046A90039EE9545F538D3E54F9400E54E6480948D
:1046B900804025900024E0FEA3E0FFE54F2FFFE5B1
:1046C9004E3EFEEF249CFFEE34FFFEC3EF9541F50D
:1046D9003BEE9540F53A801B900024E0FEA3E0FFF5
:1046E900EF249CFFEE34FFFEC3EF9541F53BEE95B9
:1046F90040F53A201703024941AE43AF447C007D9F
:1047090002121E12D3E5399FEE6480F8E538648001
:104719009840289001EAE0FFEF20E5067549007509
:1047290048000549AF49EFD394504003754950E516
:1047390049C3940A405453080E804FAE43AF447C9A
:10474900007D02121E12C3E49FFFE49EFEC3E539F9
:104759009FEE6480F8E53864809850289001EAE07B
:10476900FFEF20E4067549007548000549AF49EF98
:10477900D394504003754950E549C3940A400B53FB
:10478900080D8006754900754800AE43AF447C00AA
:104799007D02121E12D3E53B9FEE6480F8E53A6470
:1047A900809840289001EAE0FFEF20E7067547006E
:1047B9007542000547AF47EFD39450400375475002
:1047C900E547C3940A406153080B805CAE43AF448C
:1047D9007C007D02121E12C3E49FFFE49EFEC3E526
:1047E9003B9FEE6480F8E53A6480985035D3E54103
:1047F9009400E5406480948040289001EAE0FFEF4E
:1048090020E6067547007542000547AF47EFD39488
:10481900504003754750E547C3940A400B530807B6
:104829008006754700754200AF39AE3812000E8E0A
:104839003C8F3DC37428953DFFE4953CFEEF78021B
:10484900C333CE33CED8F9FFAD487C00C3EF9DF515
:104859003FEE9CF53EC3E53E648094805006753E6C
:1048690000753F00E549C39450501DAF497E007C57
:10487900007D7F121E007C007D50121E12EF2480E5
:10488900FFEF64FFF5FA8027C3E53D9428E53C6412
:104899008094805017E548C394A050100548C3E59B
:1048A9003E648094804008853FFA800375FA00AF22
:1048B9003BAE3A12000E8E3C8F3DC37428953DFFE6
:1048C900E4953CFEEF7802C333CE33CED8F9FFAD81
:1048D900427C00C3EF9DF53FEE9CF53EC3E53E6487
:1048E9008094805006753E00753F00E547C394509B
:1048F900501DAF477E007C007D7F121E007C007D2D
:1049090050121E12EF2480FFEF64FFF5FE803BC3B7
:10491900E53D9428E53C648094805017E542C394B2
:10492900A050100542C3E53E64809480401C853F39
:10493900FE801775FE00801275490075480075479D
:104949000075420075FA0075FE00E508C454F0FFD1
:10495900EF240FFF9001EAEFF09001EAE0FF8FA04A
:01496900222B
:106763004310000043D8000044A20000451100007C
:1067730045B400004622000000C700C70002000A1B
:106783000E0F03840E0F03840001000100000000BC
:086793000000000000000000FE
:10674F00011400011663011200011700011A00C1A4
:03675F000CC18BDF
:03000300025E1585
:105E1500C0E0C083C08263A201C083C082C0D075C8
:105E2500D000C006C007200B4F200C4CD2B330B3B6
:105E3500020512051AAF1AC3EF64809488401CAF9F
:105E450017EF3395E0FE74402FF58274003EF5831D
:105E5500E512F07512000517751A00E5122512F501
:105E650012C3E51764809484404F751700D20C90D7
:105E75000048E0FF8F128041200B3E300C3BE512BD
:105E85002512F512A2D792B3051AAF1AC3EF648093
:105E95009488401A0517AF17EF3395E0FE74482F25
:105EA500F58274003EF583E0FF8F12751A00C3E595
:105EB50017648094A04002D20BD007D006D0D0D072
:0D5EC50082D08363A201D082D083D0E0326E
:104E6200900048E552F0A3E553F0E54F2484FFE5B6
:104E72004E3403FE90004AEEF0A3EFF090004CE5B2
:104E820045F0A3E546F0E5412484FFE5403403FE06
:104E920090004EEEF0A3EFF0E50B2484FFE50A3418
:104EA20003FE900050EEF0A3EFF0900022E0FEA38C
:104EB200E0FF900052EEF0A3EFF0900024E0FEA39A
:104EC200E0FF900054EEF0A3EFF0900028E0FEA384
:104ED200E0FF900056EEF0A3EFF0900058E543F0AB
:104EE200A3E544F030170B90005AE4F0A37401F0EC
:104EF200800890005AE4F0A3E4F0900015E0FFEF80
:104F02003395E0FE90005CEEF0A3EFF0900014E029
:104F1200FFEF3395E0FE90005EEEF0A3EFF090001D
:104F220013E0FFEF3395E0FE900060EEF0A3EFF0A8
:104F3200900012E0FFEF3395E0FE900062EEF0A3E6
:104F4200EFF0900011E0FFEF3395E0FE900064EE89
:104F5200F0A3EFF0900041E0F516900040E4F0A3DA
:104F62007463F0C3E516648094884003025047C31B
:104F7200E516648094805003025047900042E0F5A9
:104F820018A3E0F519AF16EF3395E0FEEF25E0FF29
:104F9200EE33FE747B2FF58274673EF583E493FE55
:104FA200740193FFD3E5199FEE6480F8E5186480DD
:104FB200984021AF16EF3395E0FEEF25E0FFEE3388
:104FC200FE747B2FF58274673EF583E493F51874C3
:104FD2000193F519AF16EF3395E0FEEF25E0FFEEF2
:104FE20033FE748B2FF58274673EF583E493FE746F
:104FF2000193FFC3E5199FEE6480F8E51864809879
:105002005021AF16EF3395E0FEEF25E0FFEE33FEC1
:10501200748B2FF58274673EF583E493F51874015F
:1050220093F519AF16EF3395E0FEEF25E0FFEE336F
:10503200FE74222FF58274003EF583E518F0A3E595
:1050420019F0124D37E516B40805A217B3921722CC
:03002B00025ED2A0
:105ED200C0E0C0F0C083C08263A201C083C082C0A0
:105EE200D075D000C000C001C002C003C004C0050C
:105EF200C006C007C2CF75A61E75A6E11509AF0977
:105F0200EF705E75090490003AE0FEA3E0FFEF8EA9
:105F1200F0121FE15F3A00005F3F00015F440002A0
:105F22005F4900035F4E00045F5300055F5800069F
:105F32005F5D000700005F6012618F80211262398D
:105F4200801C1264168017125B54801212679B80A9
:105F52000D12575F80081258668003125969124663
:105F620089D007D006D005D004D003D002D001D00A
:105F720000D0D0D082D08363A201D082D083D0F06F
:035F8200D0E0323A
:030023000266333F
:10663300C0E0C0F0C083C08263A201C083C082C037
:10664300D075D000C000C001C002C003C004C005A3
:10665300C006C007C2AC30981AC298E599B43F038C
:10666300125052E599B4210B12539ED20DD20ED281
:106673000FD210C299D2ACD007D006D005D004D027
:1066830003D002D001D000D0D0D082D08363A20146
:09669300D082D083D0F0D0E032B7
:03000B00025F850C
:105F8500C0E0C0F0C083C08263A201C083C082C0EC
:105F9500D075D000C000C001C002C003C004C00558
:105FA500C006C007758A00758C4C75A61E75A6E1DE
:105FB5000514AF14C3EF6480948A4016300B137533
:105FC5001400751700751A00C20CC20B7512001269
:105FD5004E62E51375F007121D86AFF0EF701E12C5
:105FE5003B76301104D20DD210E55A60073011040A
:105FF500D20ED20F12002E124C88124D441513AF3B
:1060050013EF700C75134ED211301104D20ED20F4E
:10601500D007D006D005D004D003D002D001D000DF
:10602500D0D0D082D08363A201D082D083D0F0D0EB
:02603500E03257
:10217B00758FFF758921758DFF438780759850D2B8
:10218B008CD28ED2CA75CB4C75CA0043B81143B7EB
:10219B0021D28875D90243D84075DA4275DE42C226
:1021AB00117513467509017F021256A91256F67561
:1021BB005B00900040E4F0A37463F020A003126571
:1021CB00B975A8B375A707E55A70FC900036E0FC0B
:1021DB00A3E0FDEC121ACD7B007A00792078411236
:1021EB0019AD7B007A00793478C31217B39001CA0A
:1021FB00E0F8A3E0F9A3E0FAA3E0FB1218A4900027
:10220B001E121F5E900038E0FCA3E0FDEC121ACD0D
:10221B007B007A00792078411219AD7B007A007926
:10222B00B478C21217B39001CAE0F8A3E0F9A3E0A7
:10223B00FAA3E0FB1218A490001A121F5E90001173
:10224B00E0FCEC121AD27B007A0079B478441219B4
:10225B00ADC004C005C006C007900012E0FCEC1234
:10226B001AD27B007A0079C078411219ADA804A963
:10227B0005AA06AB07D007D006D005D0041217B3BA
:10228B00C004C005C006C007900010E0FCEC121A99
:10229B00D27B007AC079A878471219ADA804A9059A
:1022AB00AA06AB07D007D006D005D0041217B390FF
:1022BB000044121F5E900014E0FFEF3395E0FEFD2B
:1022CB00FCEF2409FFEE3400FEED3400FDEC34008E
:1022DB00FC7B0C7A007900780012669CA804A90597
:1022EB00AA06AB07900015E0FFEF3395E0FEFDFC6F
:1022FB00EF24D0FFEE3407FEED3400FDEC3400FC90
:10230B00EB2FFFEA3EFEE93DFDE83CFC7B077A0044
:10231B0079007800121E5E7B047A00790078001237
:10232B00669CC004C005C006C007900015E0FFEF17
:10233B003395E0FEFDFC7B6F7A0179007800121E6D
:10234B005ED003D002D001D000C3EF9BFFEE9AFE0C
:10235B00ED99FDEC98FCC004C005C006C0079000C9
:10236B0014E0FFEF3395E0FEFDFC7B137A0179005F
:10237B007800121E5E7B097A007900780012669C49
:10238B00A804A905AA06AB07D007D006D005D00430
:10239B00EB2FFBEA3EFAE93DF9E83CF8900013E03D
:1023AB00FFEF3395E0FEFDFCEB2FFFEA3EFEE93D30
:1023BB00FDE83CFCEF247AF511EE34E0F510ED343A
:1023CB0000F50FEC3400F50E900028E0FEA3E0FFC3
:1023DB00EF64014E70487B017A007908C003C0029C
:1023EB00C0017B017A007968900193EBF0A3EAF0CE
:1023FB00A3E9F0AF11AE10AD0FAC0E900196121F0A
:10240B005E900044E0FCA3E0FDA3E0FEA3E0FF90A0
:10241B00019A121F5ED001D002D003123FC190006F
:10242B0028E0FEA3E0FFEF4E60030226007B017A5B
:10243B00007908C003C002C0017B017A0079689063
:10244B00010BEBF0A3EAF0A3E9F0AF11AE10AD0F67
:10245B00AC0E90010E121F5E900044E0FCA3E0FD59
:10246B00A3E0FEA3E0FF900112121F5ED001D00289
:10247B00D0031229D590001AE0FCA3E0FDA3E0FEE7
:10248B00A3E0FF12525E7B547AE379457840121831
:10249B00A4C004C005C006C007900016E0FCA3E072
:1024AB00FDA3E0FEA3E0FF125274A804A905AA063F
:1024BB00AB07D007D006D005D0041218A4C004C0B7
:1024CB0005C006C007900068E0FCA3E0FDA3E0FE9A
:1024DB00A3E0FF12525EA804A905AA06AB07D0071A
:1024EB00D006D005D0041218A4C004C005C006C085
:1024FB0007AF11AE10AD0FAC0EC004C005C006C0C7
:10250B00077FAB7EAA7D2A7C3C900044E0F8A3E0D9
:10251B00F9A3E0FAA3E0FB1217B3900146121F5E7A
:10252B00D007D006D005D004120C7DC004C005C066
:10253B0006C007AF11AE10AD0FAC0EC004C005C086
:10254B0006C0077FAB7EAA7D2A7CBC900044E0F8D6
:10255B00A3E0F9A3E0FAA3E0FB1217B39001461234
:10256B001F5ED007D006D005D004120C7DD003D04F
:10257B0002D001D0001217AF7B007A007987784325
:10258B001219ADA804A905AA06AB07D007D006D02F
:10259B0005D0041217B37B007A00797A78441218AD
:1025AB00A4121B068E0C8F0DAC0CAD0DEC121ACDBC
:1025BB00C004C005C006C00790003CE0FEA3E0FFCE
:1025CB00EF7802C333CE33CED8F9FF74632FF58285
:1025DB0074673EF583121F2ED007D006D005D004AA
:1025EB001218A47B007A00797A78441219AD121B69
:1025FB00068E1B8F1C900028E0FEA3E0FFEF640209
:10260B004E7014900068121F6A3F82D0E59000084C
:10261B00121F6A40C39DB2900028E0FEA3E0FFEFBB
:10262B0064034E7014900068121F6A3F3566CF909A
:10263B000008121F6A40A73B64900028E0FEA3E04D
:10264B00FFEF64044E7014900068121F6ABF018F75
:10265B00C5900008121F6A40953F7D900028E0FE50
:10266B00A3E0FFEF64054E7014900068121F6A3EE2
:10267B00C44D01900008121F6A3FB91687900028BD
:10268B00E0FEA3E0FFEF64064E7014900068121F8B
:10269B006A3F32B6AE900008121F6A401F2B0290A1
:1026AB000028E0FEA3E0FFEF64074E701490006873
:1026BB00121F6A00000000900008121F6A40BC7ACB
:1026CB00E1900028E0FEA3E0FFEF64084E706790F6
:1026DB000032E0FCA3E0FDEC121ACD7B007A00790E
:1026EB002078411219AD9001CAE0F8A3E0F9A3E0FC
:1026FB00FAA3E0FB1218A4900008121F5E9000349E
:10270B00E0FCA3E0FDEC121ACD7B007A0079207877
:10271B00411219AD7B007A0079B478C21217B390CD
:10272B0001CAE0F8A3E0F9A3E0FAA3E0FB1218A4B6
:10273B00900068121F5E900028E0FEA3E0FFC3EF3D
:10274B009409EE648094804003022854900044E086
:10275B00FCA3E0FDA3E0FEA3E0FFC004C005C006A0
:10276B00C007AF11AE10AD0FAC0E9001B6121F5ECD
:10277B00D007D006D005D004124389900170121FE8
:10278B005E7B017A00790CC003C002C0017B017A29
:10279B0000790090016DEBF0A3EAF0A3E9F0900053
:1027AB0008E0FCA3E0FDA3E0FEA3E0FF90017412A0
:1027BB001F5E900068E0FCA3E0FDA3E0FEA3E0FF3A
:1027CB00900178121F5ED001D002D0031231DC9041
:1027DB000028E0FEA3E0FFEF4E705A900000E0FCF3
:1027EB00A3E0FDA3E0FEA3E0FF12525E7B007A5054
:1027FB0079C778451218A4C004C005C006C007905D
:10280B0000D0121F6A48B98C00D007D006D005D073
:10281B0004126379A804A905AA06AB07900000E08F
:10282B00FCA3E0FDA3E0FEA3E0FF1217AF900004B2
:10283B00121F5E8014900000E0FCA3E0FDA3E0FEFD
:10284B00A3E0FF900004121F5E900028E0FEA3E0BF
:10285B00FFEF64094E705C90002EE0FCA3E0FDECF2
:10286B00121ACD7B007A00792078411219AD9001B4
:10287B00CAE0F8A3E0F9A3E0FAA3E0FB1218A490D6
:10288B00000C121F5E900030E0FCA3E0FDEC121A6E
:10289B00CD7B007A00792078411219AD9001CAE006
:1028AB00F8A3E0F9A3E0FAA3E0FB1218A49000044C
:1028BB00121F5E900028E0FEA3E0FFEF640A4E704B
:1028CB005C90002AE0FCA3E0FDEC121ACD7B007AB1
:1028DB0000792078411219AD9001CAE0F8A3E0F914
:1028EB00A3E0FAA3E0FB1218A490000C121F5E9059
:1028FB00002CE0FCA3E0FDEC121ACD7B007A0079F2
:10290B002078411219AD9001CAE0F8A3E0F9A3E0D9
:10291B00FAA3E0FB1218A4900004121F5E9001CAE8
:10292B00E0F8A3E0F9A3E0FAA3E0FB90000CE0FCD5
:10293B00A3E0FDA3E0FEA3E0FF1219AD7BCD7ACCA3
:10294B00794C783D1217B37B007A007920784112CD
:10295B0018A4121B068E528F539001CAE0F8A3E005
:10296B00F9A3E0FAA3E0FB900004E0FCA3E0FDA3D5
:10297B00E0FEA3E0FF1219AD7BCD7ACC794C783D0C
:10298B001217B37B007A00792078411218A4121B1E
:10299B00068E4E8F4F7F007E007D207C419000681D
:1029AB00E0F8A3E0F9A3E0FAA3E0FB1218A490016E
:1029BB00CAE0F8A3E0F9A3E0FAA3E0FB1219AD1209
:0A29CB001B068E0A8F0B0221D22298
:10564200EFC0E0C283740F12567774301256817421
:1056520005125677743012568174011256777430DF
:105662001256817401125677D0E014600274084415
:105672002012568F227D000000DDFCD5E0F7225477
:10568200F053800F4280C282D283C28322C28280C0
:1056920002D282C0E012569DD0E0C454F053800F73
:1056A2004280D283C283221256421256DB74061201
:1056B200568F1256DB740E12568F1256DB7401127D
:1056C200568F1256DB744012568F1257281256DB31
:1056D200748012568F12570822740A12567722EFDC
:1056E200C0E01256DBD0E0125693221256DB74024F
:1056F20012568F221256DB740112568F221256DB7B
:10570200740E12568F221256DB740C12568F22120E
:1057120056DB740F12568F22EFC0E01256DBD0E038
:10572200448012568F229057377E28E493FF1256F8
:10573200E1A3DEF7220004040E0E1F1F00001F1F4C
:105742000E0E04040000101C1F1C100000000107B4
:0D5752001F070100000E11171917110E009E
:1067EA007A107B00EE6BFB8BF053F080ABF033EF4B
:0867FA0033FFEE33FEDAEE225C
:1064A9009001E1EEF0A3EFF09001E1E0FEA3E0FF3F
:1064B9007C037DE8121E12EF2430F5993099FDC254
:1064C900999001E1E0FEA3E0FF7C037DE8121E1232
:1064D9007E007F64CFCDCFCECCCE121E12EF2430FA
:1064E900F5993099FDC2999001E1E0FEA3E0FF7CA6
:1064F900007D64121E127E007F0ACFCDCFCECCCE96
:10650900121E12EF2430F5993099FDC2999001E1DC
:10651900E0FEA3E0FF7C007D0A121E12AF05EF2406
:1065290030F5993099FDC2997599003099FDC29954
:01653900223F
:105052009001E37475F0A37430F020981C9001E382
:10506200E0FEA3E0FFEF4E60109001E4E024FFF0C9
:105072009001E3E034FFF080E1C298AF99EF121F94
:10508200BB50D56150E16250ED6350F5645101654A
:10509200510D66511967512568513169513D6A5167
:1050A200496B51556C51616D516D6E517B6F5183DE
:1050B2007051917151997251A77351AF7451C27568
:1050C20051D07651DE7751EC7851FA7952087A0054
:1050D200005215900022E0FEA3E0FF1264A9229084
:1050E2000024E0FEA3E0FF1264A922AF44AE431203
:1050F20064A922900028E0FEA3E0FF1264A9229096
:10510200002AE0FEA3E0FF1264A92290002CE0FE38
:10511200A3E0FF1264A92290002EE0FEA3E0FF129A
:1051220064A922900030E0FEA3E0FF1264A922905D
:105132000032E0FEA3E0FF1264A922900034E0FEF8
:10514200A3E0FF1264A922900036E0FEA3E0FF1262
:1051520064A922900038E0FEA3E0FF1264A9229025
:10516200003AE0FEA3E0FF1264A922E50D2488FFC5
:10517200E50C3413FE1264A922AF46AE451264A9AF
:1051820022E5412484FFE5403403FE1264A922AFE4
:1051920053AE521264A922E54F2484FFE54E340334
:1051A200FE1264A922AF0BAE0A1264A922301708BC
:1051B2007F017E001264A9227F007E001264A92270
:1051C200900010E0FFEF3395E0FE1264A9229000F8
:1051D20011E0FFEF3395E0FE1264A922900012E085
:1051E200FFEF3395E0FE1264A922900013E0FFEF77
:1051F2003395E0FE1264A922900014E0FFEF33958C
:10520200E0FE1264A922900015E0FFEF3395E0FE64
:035212001264A97A
:015215002276
:10653A009001D6E4F0A3E4F09001D87475F0A37446
:10654A0030F09001DAE4F09001DAE0FFD3EF6480F2
:10655A009483505220981C9001D8E0FEA3E0FFEFEC
:10656A004E60109001D9E024FFF09001D8E034FF8A
:10657A00F080E1C2989001D6E0FEA3E0FF7C007DA6
:10658A000A121E00AD997C00EF2DFFEE3CFEEF24AF
:10659A00D0FFEE34FFFE9001D6EEF0A3EFF09001AB
:0E65AA00DAE004F080A19001D6E0FEA3E0FF4D
:0165B80022C0
:10539E009001E57475F0A37430F020981C9001E52F
:1053AE00E0FEA3E0FFEF4E60109001E6E024FFF078
:1053BE009001E5E034FFF080E1C298AF99EF121F43
:1053CE00BB540F61541E62542D63543C64544B65A0
:1053DE00545A6654696754786854876954966A5467
:1053EE00A56B54B46C54C36D54D27454D87554E434
:1053FE007654F07754FC7855087955147A00005598
:10540E001F12653A900022EEF0A3EFF0124D3722F4
:10541E0012653A900024EEF0A3EFF0124D372212EF
:10542E00653A900026EEF0A3EFF0124D372212658A
:10543E003A900028EEF0A3EFF0124D372212653AA3
:10544E0090002AEEF0A3EFF0124D372212653A903B
:10545E00002CEEF0A3EFF0124D372212653A9000B9
:10546E002EEEF0A3EFF0124D372212653A90003077
:10547E00EEF0A3EFF0124D372212653A900032EEA5
:10548E00F0A3EFF0124D372212653A900034EEF091
:10549E00A3EFF0124D372212653A900036EEF0A3CC
:1054AE00EFF0124D372212653A900038EEF0A3EF6E
:1054BE00F0124D372212653A90003AEEF0A3EFF05B
:1054CE00124D3722A217B392172212653A9000108E
:1054DE00EFF0124C332212653A900011EFF0124C9D
:1054EE00332212653A900012EFF0124C33221265FD
:1054FE003A900013EFF0124C332212653A900014DA
:10550E00EFF0124C332212653A900015EFF0124C68
:01551E003359
:01551F002269
:1017AC00021B72E86480F8E933E83360110460F0DE
:1017BC00ED33EC337009E8FCE9FDEAFEEBFF2204A3
:1017CC0060DED3EB9FEA9EE99DE8C2E78CF0C2F79E
:1017DC0095F0400CE8CCF8E9CDF9EACEFAEBCFFB6A
:1017EC00121B3D85D0F05804700320D5B3E804706B
:1017FC00075002B2D5021B7C92D5EC0460F7E4CC06
:10180C00C0E0C398F8603B94186008400DD0E0FB32
:10181C00021B54E4FBFAC9FC8028E830E406E4C956
:10182C00FBE4CAFCE830E305E4C9CACBFCE8540786
:10183C006010F8C3E913F9EA13FAEB13FBEC13FC91
:10184C00D8F130F52FC3E49CFCEF9BFFEE9AFEED34
:10185C0099FDD0E0FBEF4E4D4C701222DB03021BC6
:10186C0079EC2CFCEF33FFEE33FEED33FDED30E77E
:10187C00EB021B54EF2BFFEE3AFEED39FDD0E0FBF3
:10188C0050130BBB0003021B7CED13FDEE13FEEF9C
:08189C0013FFEC13FC021B54C6
:1018A400EC4D6011E8497017ED33EC3304600DE43E
:1018B400FCFFFEFD22E933E8330470F8021B7212C8
:1018C4001B3D58046009E4CC2481500628500902C9
:1018D4001B7C284003021B79C0E0EB4A7044B980AA
:1018E40006D0E0FB021B68EF4E701CBD8008EBFFC6
:1018F400EAFEE9FD80EBE98DF0A4FEE5F002198D26
:10190400E9CDF9EAFEEBFFEF89F0A4FCE5F0CE891E
:10191400F0A42EFFE435F0CD89F0A42DFEE435F0DB
:101924008067EF4E7005BD80D780C3EF8BF0A4AC09
:10193400F0EE8BF0A42CFCE435F0F8EF8AF0A42C44
:10194400E5F038FCE433CB8DF0A42CFCE5F03BF857
:10195400EE8AF0A42CFCE5F038F8E433CF89F0A447
:101964002CFCE5F038CF3400CE89F0A42FFFE5F04D
:101974003EFEE433C98DF0A42EFEE5F039CD8AF0A5
:10198400A42FFFE5F03EFEE43DFD33D0E0FB50071D
:101994000BBB000F021B7CEC2CFCEF33FFEE33FE81
:0619A400ED33FD021B54AF
:1019AA00021B7CEC5D046005E859047003021B729B
:1019BA00121B3D580460F6EC4860F2EC7004FDFE20
:1019CA00FF22C860DB2481C85009C3986002500610
:1019DA00021B799850CAF582E9294B4A7005AB82F5
:1019EA00021B6875F0007C1A7880C3EF9BEE9AEDB3
:1019FA0099400DC3EF9BFFEE9AFEED99FDE842F088
:101A0A00DC23ACF0D0E0FFD0E0FED0E0FDAB8220DA
:101A1A00E7101BEB60BAEC2CFCEF33FFEE33FEED64
:101A2A0033FD021B54E803F830E705C0F075F000F7
:101A3A00EF2FFFEE33FEED33FD40B830E7C280AA48
:101A4A0074F8CC6480CCC86480C8F582046043C34F
:101A5A00EB9FF5F0EA9E42F0E99D42F0E89C45F0E2
:101A6A0060305018E5825FFFE582F42B5582FB5007
:101A7A00210ABA001D09B90019088016E5825BFB24
:101A8A00E582F42F5582FF50090EBE00050DBD00F8
:101A9A00010CC3EB9FF5F0EA9E42F0E99D42F0E8A3
:0D1AAA009C45F06007CC4820E701B3EC221A
:101AB700ED33EC33600A047003BD8004ECB2E7FC3D
:011AC70022FC
:101AC80075F020800E75F010800575F0087D007E99
:101AD800007F003392D530D503121EADEC33401091
:101AE800EF33FFEE33FEED33FDEC33FCD5F0ED22A2
:0E1AF800E5F0247EA2D513CC92E7CDCEFF22DE
:101B0600EDD2E7CD33EC3392D524814006E4FFFED7
:101B1600FDFC22FCE4CFCECDCC24E0501174FF8036
:101B2600EDC3CC13CCCD13CDCE13CECF13CF0470D3
:071B3600F030D5DE021EAD08
:1036F300E56724DBF582E43400F583E00567229077
:1037030000D83009039000DBE475F001121F9B021F
:103713001DA82002E97F2ED2028018EF540F2490B7
:10372300D43440D4FF30060BEF24BFB41A00500347
:103733002461FFE56860021568056BE56B7002059F
:103743006A30090E9000D8E475F001121F9BEF0256
:103753001DEE0267C37403D2098003E4C209F5674F
:103763009000D8121FB2E4F568F56AF56BE568605E
:10377300077F2012373680F57569FFC203C202C284
:1037830004C205C207C208C20A123702FF700D3015
:1037930009057F00123747AF6BAE6A22B4255FC2BB
:1037A300D5C206123702FF24D0B40A00501A75F0AE
:1037B3000A786830D50508B6FF0106C6A426F620A8
:1037C300D5047002D20580D924CFB41A00EF500477
:1037D300C2E5D206023A39D20380C6D20280C0D2F1
:1037E3000480BCD2D580BAD20780B47F201237368A
:1037F3002004077401B5680040F11236F3FF123755
:1038030036023770D20AD20880951236F3FB12368D
:10381300F3FA1236F3F94A4B700679377A3B7BFF9A
:1038230020042EE568602A7E008E82758300121DB7
:10383300C160060EEE656970F0C2D5EBC0E0EAC068
:10384300E0E9C0E0EE123A9AD0E0F9D0E0FAD0E035
:10385300FB121DA8FF60AAEBC0E0EAC0E0E9C0E0EC
:10386300123736D0E02401F9D0E03400FAD0E0FB7F
:10387300E5690460DCD569D98087D20480A2123A55
:103883007C60F7E569700104121B87A969600DE587
:1038930069600914F569123B24EF60F3EA30E7022B
:1038A300F404C3995079EAF425690430E701E40488
:1038B300F569800D123A7C60C1EA05692569121B1E
:1038C30087EA900107F030E701E4256904D569042C
:1038D30020070114123A9AE4C0E0123B2490010736
:1038E300E0601320E70714F012371E802204F0D0A3
:1038F300E014C0E07F0012371EE569600712371538
:103903001569800B300703123715D0E0023770D0EA
:10391300E00480C4123A7C609EE56904121B879020
:103923000107EAF0E5692007026001042404123A62
:013933009AF9
:1039340074FF04C0E0123B2412371EE5692007021D
:103944006003123715D0E0B569E87F451237289037
:103954000107E07F2B30E7047F2DF404C0E0123729
:1039640036D0E075F00A84C0F012371FD0E0123769
:103974001F023770791080027908C208C20A8008D1
:10398400D2D5790A8004790AC2D5E569047002F5B2
:1039940069E4FAFDFEFF1236F3FC7B0820031312E0
:1039A40036F3FD7B1030020A1236F3FE1236F3FFB3
:1039B4007B20EC3382D592D55013C3E43002069FAA
:1039C400FFE49EFEE42003039DFDE49CFCE4CBF8AD
:1039D400C203EC700CCFCECDCCE824F8F870F380A1
:1039E40017C3EF33FFEE33FEED33FDEC33FCEB3363
:1039F400FB994002FB0FD8E9EB300305F8D0E0C493
:103A040048B203C0E00AEC4D4E4F78207B0070C2F0
:103A1400EAB5690040BCC0E0123A9CD0F0D0E02086
:103A24000304C4C0E0C4B203C0F012371FD0F0D501
:103A3400F0EB023770121FBB380D5339785837DE5C
:103A44004C37DA42397C4F39844439844937F3435B
:103A5400398A5538B7463917453881473B57503767
:103A6400E22D37E62E38092B37EA233807203B406E
:103A74002A37A24800003801E569B4FF03756906D6
:103A84001236F3FC1236F3FD1236F3FE1236F3FF50
:103A9400900100021BC4790AA2D52005143007093D
:103AA400B910020404B9080104A2D5200802500187
:103AB400042004689204B568005034C0E07F2030CC
:103AC40005197F30A20472087207500F123AF3C22C
:103AD40004C208C207C20A7F30800F300703E9C05E
:103AE400E0123736300703D0E0F9D0E0B568CC30C7
:103AF40007177F30B9100C1237367F583006077F0E
:103B0400788003B908031237363004057F2D023755
:103B1400367F20200AF87F2B2008F322920480CFDE
:103B24007F00B40700500B2400F582E43401F583D0
:103B3400E0FF22286E756C6C2900D2031236F33034
:103B440003F8C203786830D50108F60237A22D5075
:103B54004349581236F32403B405004001E4903B72
:103B64005293123727743A123727D2057568040224
:023B740039789E
:0D683500ED33EC3360065004EC6480FC226F
:1060E300021B7222EDA2E7D2E7F9EC3340F260F330
:1060F300B4FF08ED547F70E8021B7CF82481C2E0F2
:10610300C0E0F40428FAC313FCED92E7FD9000CC41
:10611300121F5EEEA2E7E9BA7F02C31334009400B4
:10612300FA75F091A4E5F013F494FE8AF0A433E534
:10613300F033248CD313FDE492E7FE7F007C3F759C
:106143008302ECC0E0F8EDC0E0F9EEC0E0FAEFC086
:10615300E0FB8583F09000CC121F0685F0831219B3
:10616300ADD0E0FBD0E0FAD0E0F9D0E0F81217B3FD
:10617300ED6480FD30E7011CD583C7ED33CC33F8E4
:0C618300D0E0A2E71328C313CC13FD22C8
:106379009000CC121F5E9000D0E0F8A3E0F9A3E0F2
:10638900FAA3E0FB9000CCE0FCA3E0FDA3E0FEA3B0
:10639900E0FF1219AD1255409000CC121F5E90001B
:1063A900D0E030E7599000CCE0FCA3E0FDA3E0FE8B
:1063B900A3E0FFECC0E0EDC0E0EEC0E0EFC0E0E438
:1063C900FFFEFDFC9000CCE0F8A3E0F9A3E0FAA3FE
:1063D900E0FB121A4A7BDB600250087A0F79497890
:1063E9004080067A0F794978C0D0E0FFD0E0FED02E
:1063F900E0FDD0E0FC1217B39000CC121F5E9000B4
:0D640900CCE0FCA3E0FDA3E0FEA3E0FF2239
:105216003A70FA83BCAAE9E43E81E0F8BF9DE9E66C
:105226003F80000039283C1ABB9969663DA335E3E7
:10523600BF255DE73FC90FDB418DDBCCC44936EEA8
:1052460045C9913FC5B0F83D3F800000C317F5340E
:10525600452FFA73C60AFDDD12531F04A2E1920020
:105266001420E0159052167404121CC98030125393
:105276001F30E102B20020E0EBA883A9829000CCA7
:10528600121F5E8982888390522A7404121CC98573
:1052960082F09000CC121F2285F0821218A4ED4CE9
:1052A6006007300004EC6480FC2212531FC0E0A8A3
:1052B60083A9829000CC121F5E8982888390524E09
:1052C6007403121CC98582F09000CC121F2285F04F
:1052D600821218A49000CCE0CCF0A3E0CDF0A3E0BD
:1052E600CEF0A3E0CFF090523E7403121CC9D082D8
:1052F6008582F09000CC121F2285F082E58230E094
:10530600071219ADB2008096EFCBFFEECAFEEDC9CB
:10531600FDECC8FC1219AD8085ED33EC547FCC331F
:10532600920024605007D0E0D0E0021B727B837AA3
:10533600F97922783E1218A4EDF933ECF83324817A
:105346005011EFFBEEFA121B06121AC8ECB2E7FC7C
:105356001217B3ED33EC33602F2403F8C313FCEDBF
:1053660092E7FDE82481E4501FECF8EDF9EEFAEF40
:10537600FB121B06EF04C2E0FCF582121AD2ECB255
:10538600E7FC1217B3E58203FAED33EC336007143A
:0853960013FCED92E7FDEA2291
:10552000BE1249253E4CCCCDBEAAAAAB3F8000009E
:105530003E7ADBB03EED63383F24BC7D3F490FDB54
:10554000ED33ECC2E7CC339200B4FF13ED547F602F
:1055500003021B727FDB7E0F7DC97C3F025635C282
:1055600001C3947F401E7007EDD2E794904015EF81
:10557000FBEEFAEDF9ECF87F007E007D807C3F12B7
:1055800019ADD201ED33EC33248430E705E4C0E0FB
:10559000806B04FAEDD2E754F0C333DAFD540734DC
:1055A000002323C0E0CCC0E0F8EDC0E0F9EEC0E09D
:1055B000FAEFC0E0FBE4121AD2EC24FEFC9000D417
:1055C000121F5E1218A47B007A007980783F1217B0
:1055D000B39000D4E0B2E7CCF0A3E0CDF0A3E0CEEE
:1055E000F0A3E0CFF0D0E0FBD0E0FAD0E0F9D0E0DB
:1055F000F81217B39000D4121F221219AD9000D4E4
:10560000121F5E9055207403121CC99000D4121F03
:10561000221218A4D0E0600F242CF582E43455F552
:1056200083121F2E1217B330010B7BDB7A0F79C95F
:1056300078BF1217B3ED33EC336006ECA20092E7AB
:02564000FC224A
:105A64009000CC121F5E74FFFFFEFDFC9000CCE0A2
:105A7400F8A3E0F9A3E0FAA3E0FBC3121EBB60386D
:105A84007F807E967D187C4B9000CCE0F8A3E0F9F3
:105A9400A3E0FAA3E0FB121A4A6002501B7F807E47
:105AA400967D187CCB9000CCE0F8A3E0F9A3E0FA53
:105AB400A3E0FB121A4A500F9000CCE0FCA3E0FDD7
:105AC400A3E0FEA3E0FF229000CCE0FCA3E0FDA352
:105AD400E0FEA3E0FF121B069000D0121F5E9000B0
:105AE400D0E0FCA3E0FDA3E0FEA3E0FFEC121AC8A3
:105AF400C8ECC8C9EDC9CAEECACBEFCB9000CCE064
:105B0400FCA3E0FDA3E0FEA3E0FF1217AFE4FBFA61
:105B1400F9F8121A4A602640249000D0E0FCA3E071
:105B2400FDA3E0FEA3E0FFEF24FFFFEE34FFFEED54
:105B340034FFFDEC34FFFC9000D0121F5E9000D0C7
:105B4400E0FCA3E0FDA3E0FEA3E0FFEC121AC822F0
:101B3D00E9D2E7C933E833F892D5EDD2E7CD33ECEE
:071B4D0033FC5002B2D52267
:101B5400EC30E7100FBF000C0EBE00080DBD0004F2
:101B64000BEB6014A2D5EB13FCED92E7FD2274FF9E
:101B7400FCFDFEFF22E480F8A2D574FF13FC7D80F7
:031B8400E480EF0B
:101B8700F920E73624F950037907E4F42402FBE54A
:101B970082158270021583DBF6E024FB501BE96097
:101BA70014E4F0E582158270021583E004F0B40AAC
:0D1BB70008E4F0D9EE7401F00A22C2D52234
:101BC400ED33EC3392D5FA602AB4FF33EDC2E77BF0
:101BD400FF60067A1B79E9E4227A1B79F220D504A6
:101BE4007A1B79ED224E614E002B494E46002D4959
:101BF4004E4600E47A08F0A3DAFC7B00740722C0A6
:101C040083C082ECC0E0EDC0E0EEC0E0EFC0E0EAEB
:101C140075F010A4CAABF075F04DA42BFBE435F0BD
:101C2400FCEA2410FAEB34C5FBEC34D9FCEDC2E732
:101C3400FF75F056A4F42411C5F0F434C58FF0A454
:101C44002AE5F03BE43CF020E714121D46D0E0FF07
:101C5400D0E0FED0E0FDD0E0FC1219AD8014F40415
:101C6400121D46D0E0FFD0E0FED0E0FDD0E0FC1233
:101C740018A4D082D083E0FAEDD2E7CD33EC33243C
:101C840082FBE4C3CF33CFCE33CECD33CD33DBF3BE
:101C94007B0775F00A846004F0A31B0AE5F0F0A347
:101CA4008FF0740AA4FFACF08EF0740AA42CFEAC7E
:101CB400F050010C8DF0740AA42CFDE435F0F0A36F
:051CC400DBDE740722C5
:101CC900C0E0EFFBEEFAEDF9ECF81218A4D0E0F55C
:101CD900F0EFFBEEFAEDF9ECF8121F12A3A3A3A3A0
:101CE900E8C0E0E9C0E0EAC0E0EBC0E0C0F01218EB
:101CF900A4121F2EA3A3A3A31217B3D0F0D0E0FB05
:0D1D0900D0E0FAD0E0F9D0E0F8D5F0D42217
:101D16003F8000004120000042C80000447A0000D5
:101D2600461C400047C35000497424004B18968057
:101D36004CBEBC205A0E1BCA6753C21C749DC5AE4E
:101D4600FB60065407601C2323121D74EB54386095
:101D560009121D60121D6F1218A4ECF8EDF9EEFAC7
:101D6600EFCB22EB121D6F80F1543803241C901D1B
:101D760016FE93FC0EEE93FD0EEE930ECE93FF220F
:1062F90002217BE493A3F8E493A34003F68001F21F
:1063090008DFF48029E493A3F85407240CC8C333A5
:10631900C4540F4420C8834004F456800146F6DF74
:10632900E4800B0102040810204080906722E47E7B
:10633900019360BCA3FF543F30E509541FFEE49369
:10634900A360010ECF54C025E060A840B8E493A330
:10635900FAE493A3F8E493A3C8C582C8CAC583CA5B
:10636900F0A3C8C582C8CAC583CADFE9DEE780BE13
:016762000036
:101D8600C2D530F707B2D563F0FF05F030E70CB2E5
:101D9600D5F4048463F0FF05F080018430D502F4A5
:021DA600042215
:101DA800BB010689828A83E0225002E722BBFE0239
:091DB800E32289828A83E493226C
:101DC100BB010CE58229F582E5833AF583E02250D7
:101DD10006E92582F8E622BBFE06E92582F8E22221
:0D1DE100E58229F582E5833AF583E493223B
:101DEE00BB010689828A83F0225002F722BBFE01D4
:021DFE00F322CE
:101E0000EF8DF0A4A8F0CF8CF0A428CE8DF0A42EF6
:021E1000FE22B0
:101E1200C2D5EC30E709B2D5E4C39DFDE49CFCEEEB
:101E220030E715B2D5E4C39FFFE49EFE12200EC335
:101E3200E49DFDE49CFC800312200E30D507C3E430
:061E42009FFFE49EFE225A
:101E4800C5F0F8A3E028F0C5F0F8E5821582700225
:061E58001583E038F022C2
:101E5E00E88FF0A4CC8BF0A42CFCE98EF0A42CFC23
:101E6E008AF0EDA42CFCEA8EF0A4CDA8F08BF0A4A1
:101E7E002DCC3825F0FDE98FF0A42CCD35F0FCEB00
:101E8E008EF0A4FEA9F0EB8FF0A4CFC5F02ECD39C5
:0F1E9E00FEE43CFCEAA42DCE35F0FDE43CFC2232
:10669C00C2D5E830E70FB2D5E4C39BFBE49AFAE429
:1066AC0099F9E498F8EC30E717B2D51266D21220BB
:1066BC009FE4C39BFBE49AFAE499F9E498F880030D
:1066CC0012209F30D50DE4C39FFFE49EFEE49DFD98
:0466DC00E49CFC221C
:0E1EAD00C3E49FFFE49EFEE49DFDE49CFC2246
:101EBB00EB9FF5F0EA9E42F0E99D42F0E89C45F07D
:011ECB0022F4
:101ECC00BB010789828A83021F065005E9F80221AB
:101EDC0031BBFE05E9F802213D89828A83021F127B
:101EEC00BB010789828A83021F5E5005E9F8022133
:0A1EFC0063BBFE05E9F802216F2226
:0C1F0600E0FCA3E0FDA3E0FEA3E0FF224E
:101F1200E493FC740193FD740293FE740393FF2215
:0C1F2200E0F8A3E0F9A3E0FAA3E0FB2242
:101F2E00E493F8740193F9740293FA740393FB2209
:101F3E00BB010789828A83021F225005E9F802211C
:101F4E0049BBFE05E9F802215689828A83021F2EBB
:0C1F5E00ECF0A3EDF0A3EEF0A3EFF022F6
:101F6A00A8828583F0D083D082121F81121F81122A
:101F7A001F81121F81E473E493A3C583C5F0C5834F
:101F8A00C8C582C8F0A3C583C5F0C583C8C582C8C1
:011F9A002224
:101F9B00F8E0FBA3A3E0F925F0F0E58215827002CF
:071FAB001583E0FA38F02273
:091FB200EBF0A3EAF0A3E9F02230
:101FBB00D083D082F8E4937012740193700DA3A3B5
:101FCB0093F8740193F5828883E4737402936860C9
:061FDB00EFA3A3A380DFC9
:101FE100D083D082F8E4937012740193700DA3A38F
:101FF10093F8740193F5828883E473740293B5F0C6
:0D200100067403936860E9A3A3A3A380D82D
:1067C300EFB40A07740D1267CE740A309811A899B2
:1067D300B8130CC2983098FDA899C298B811F63036
:0767E30099FDC299F599220E
:10000E00C3EE6480948040028007C3E49FFFE49EA9
:02001E00FE22C0
:10200E00BC000BBE0029EF8DF084FFADF022E4CCB6
:10201E00F875F008EF2FFFEE33FEEC33FCEE9DEC7F
:10202E00984005FCEE9DFE0FD5F0E9E4CEFD22EDC5
:10203E00F8F5F0EE8420D21CFEADF075F008EF2F0F
:10204E00FFED33FD4007985006D5F0F222C398FD00
:05205E000FD5F0EA229D
:1020630075F008758200EF2FFFEE33FECD33CDCC34
:1020730033CCC58233C5829BED9AEC99E5829840B7
:102083000CF582EE9BFEED9AFDEC99FC0FD5F0D694
:10209300E4CEFBE4CDFAE4CCF9A88222B800C1B9BE
:1020A3000059BA002DEC8BF084CFCECDFCE5F0CBFC
:1020B300F97818EF2FFFEE33FEED33FDEC33FCEB35
:1020C30033FB10D703994004EB99FB0FD8E5E4F9F0
:1020D300FA227818EF2FFFEE33FEED33FDEC33FCDD
:1020E300C933C910D7059BE99A4007EC9BFCE99AD1
:1020F300F90FD8E0E4C9FAE4CCFB2275F010EF2F16
:10210300FFEE33FEED33FDCC33CCC833C810D70715
:102113009BEC9AE899400AED9BFDEC9AFCE899F850
:0E2123000FD5F0DAE4CDFBE4CCFAE4C8F922E3
:0C213100E6FC08E6FD08E6FE08E6FF22DA
:0C213D00E2FC08E2FD08E2FE08E2FF22DE
:0D214900E6FB08E6F908E6FA08E6CBF82206
:0D215600E2FB08E2F908E2FA08E2CBF82209
:0C216300ECF608EDF608EEF608EFF622A8
:0C216F00ECF208EDF208EEF208EFF222AC
:00000001FF
